:020000040000FA
:10000000C0410020F1000000F9000000D500000010
:1000100000000000000000000000000000000000E0
:10002000000000000000000000000000FD000000D3
:100030000000000000000000FF00000001010000BF
:10004000C1150000E123000000000000112A00009B
:100050000301000003010000932C0000BD2C0000F0
:10006000B929000000000000F9230000A5020020CB
:10007000292A0000D1290000E9290000A513000069
:10008000C1130000DD130000F913000000000000A0
:100090000000000003010000030100000301000054
:1000A000000000000000000000000000B107000098
:1000B00003010000630000200301000000000000B5
:1000C0000348854600F00AF900480047B9030000DC
:1000D000C041002004207146084202D0EFF309809D
:1000E00001E0EFF308807146004A10473D1500001B
:1000F0000448804704480047FEE7FEE7FEE7FEE7C6
:10010000FEE7FEE7CD280000C100000030B50B4639
:10011000014600202022012409E00D46D5409D42E1
:1001200005D31D469540491B254695404019154667
:10013000521E002DF1DC30BDF0B51FB40646002084
:1001400082B005464024019100901BE001992246AF
:100150000F46304600F0B1F8049A059B801A994189
:1001600010D310461946224600F097F8361A8F41F0
:100170000197224601200021009F00F08EF83818D8
:100180004D4100902046641E0028DFDC019B009852
:100190002946324607B0F0BDF0B51FB486B0002046
:1001A0000090019002900698069980B204900798FA
:1001B000090C02040014114307900027089D0998B8
:1001C00006913E463C4603900398A9B20204000CF7
:1001D000039004982D0C154348430021224600F05B
:1001E0005CF8C719714110340E46402CECDB3846E0
:1001F000029A00F052F8009A019B80180090594131
:1002000002980191103002904028CCDB00980BB08E
:10021000F0BD00000549064A08685043054A8018A9
:100220000860400870470149086070472C1300209F
:100230006D4EC6413930000003460B439B0703D087
:1002400009E008C9121F08C0042AFAD203E00B789B
:100250000370401C491C521EF9D27047D2B201E013
:100260000270401C491EFBD270470022F6E710B511
:1002700013460A4604461946FFF7F0FF204610BD14
:1002800030B504460020034600E05B1C934203D2D5
:10029000E05CCD5C401BF8D030BD10B5202A04DBFB
:1002A0000146203A9140002010BD914020239C1A25
:1002B0000346E3401943904010BD10B5202A04DBEB
:1002C0000846203AD040002110BD0B46D340D04014
:1002D0002024A21A91400843194610BD064C01255E
:1002E000064E05E0E36807CC2B430C3C98471034DE
:1002F000B442F7D3FFF7E8FE6C6400009C64000092
:1003000070B58C180578401C6B075B0F01D1037822
:10031000401C2A1106D10278401C03E006780E70BA
:10032000401C491C5B1EF9D12B0705D40023521E2B
:100330000DD40B70491CFAE70378401CCB1A921CB1
:1003400003E01D780D70491C5B1C521EF9D5A142BB
:10035000D8D3002070BD000003B40148019001BD56
:10036000B10C002003B40148019001BDD50D00205F
:1003700003B40148019001BD1F06002003B40148E9
:10038000019001BD0100002003B40148019001BDAE
:10039000C107002003B40148019001BDCD02002037
:1003A00003B40148019001BDEF02002003B40148ED
:1003B000019001BD5905002010B505F025F903F0A5
:1003C0002BF803F00BFC01F0B1F87D20C00002F027
:1003D000EFFF03F0F3F910BD70B5014660313F4CFB
:1003E0004A7D2270CA7D62704A780B7811021943E7
:1003F00061813022A17B125C890992068901920EEB
:100400001143A173014642314B7F0A7F190609143B
:1004100011432181014640314A7F0B7F12021A436A
:10042000E280C97EA170014641314A7E0B7E1102F5
:100430001943A180014662314B780A7819060914E4
:100440001143A1810146A0314A7F0B7F12021A435A
:10045000A2858A1C557F137F2A0612141A43E2854F
:100460000246C032567815461378320612141A43E3
:100470002286C23042780378100600141843608642
:100480001C221748FFF7D8FE2A79E97910466A79C5
:10049000090612021043AA7912041043084360634C
:1004A000082029180A7810464A78120210438A78E0
:1004B000C9781204104309060843A0630C202918C8
:1004C0000A7810464A78120210438A78C9781204D2
:1004D000104309060843E06370BD00003413002098
:1004E00043130020411C0A461378007819465378BC
:1004F0001B0219439378D2781B0419431206114347
:100500000902084370470000044A0029D16A01D05B
:10051000014300E08143D1627047000000000440C5
:10052000044A0029116B01D0014300E081431163AB
:10053000704700000000044010B5044602F032F895
:10054000154801210268890714488C4208D01449D3
:100550008C4205D013498C4202D013498C4202D1FF
:100560004069000C0DE011498C4208D010498C42C2
:1005700005D010498C4202D00F498C4209D1406904
:10058000000D0007000F04D041001046FFF7BEFD2C
:1005900010BD104610BD0000A01000200000044057
:1005A000003000400010004000800040001001407A
:1005B00000300140004001400050014070B52C4B1C
:1005C0005A69032109028A4301242A49002806D0D6
:1005D000C51FF93D0ED0FF3D012D45D129E0D86959
:1005E0002043D861D869C0013ED40846491E00287E
:1005F000F8DC39E05D6A062635435D625D6A2543B5
:100600005D620024002806D0C51FF93D05D0FF3DDE
:10061000012D05D103E0DC6902E05C6A00E09C6A20
:10062000E50103D40D46491E002DEBDCFF2001300F
:1006300019E09D6A25439D620024002806D0C51F4D
:10064000F93D05D0FF3D012D05D103E0DC6902E055
:100650005C6A00E09C6AE50103D40D46491E002D4A
:10066000EBDC0120400202435A6101F09BFF70BDA8
:100670000000044080F52000024841680122114337
:100680004160FEE70000044004480121C26A89027B
:100690000A43C26242680A434260FEE70000044027
:1006A00010B40822174B002802D0082803D005E018
:1006B000986A904301E0986A10439862986A04220D
:1006C00090439862986A08439862986A01210843A7
:1006D00098624A020C480CE0002A06D0D41FF93C6C
:1006E00005D0FF3C012C05D103E0D96902E0596A2D
:1006F00000E0996ACC0103D40446401E002CEBDCD8
:1007000010BC70470000044080F5200002480168DA
:1007100001221143016070470000074010B40E4AE7
:100720000E4B0021002806D0C41FF93C05D0FF3C29
:10073000012C05D103E0D96902E0596A00E0996A09
:10074000CC0106D41446521E002CEBDC10BC002059
:10075000704710BC0120704780F520000000044065
:1007600010B4002A07D058234B431B18DC69240B14
:1007700024031443DC610722D2018018026AFF239C
:1007800002338B401A43026210BC70475822514317
:100790000818C0698005800D7047000001220348D9
:1007A0008A4001789143017070470000A410002036
:1007B00010B500F001F810BDF8B55448006A544E69
:1007C000C007012700285DD00025B16A3846A8403F
:1007D000014254D04F4988633820294641434E484E
:1007E0000C182C20005D012804D0022831D00328E9
:1007F00045D139E029464948FFF7C8FFE18E401846
:10080000E086A18E081A02B2002A09DD01208002CA
:10081000824200DB421E29464048FFF7A1FF2EE03E
:10082000E06900282BD0A0688002800F022802D047
:10083000012805D008E0616800202031487203E0FB
:100840006168002020310872E28E1320E369216B79
:1008500014E029463148FFF7A1FF236A002B03D09B
:10086000A28E2320216B984729462C48FFF796FF3C
:10087000636A002B03D0A28E2320216B98476D1C46
:10088000022DA2DB214A106A0223810704200029DD
:100890000BDA316BC90700D01760316B890700D5BF
:1008A0001360316B490700D51060116A49070BD5F9
:1008B000B16BC90700D09760B16B890700D5936011
:1008C000B16B490700D59060116A09070CD5114931
:1008D0000C68E40700D017610C68A40700D5136109
:1008E0000968490700D51061116AC9060CD5094984
:1008F0008C68E40700D097618C68A40700D59361E9
:100900008968490700D59061F8BD000040030640A2
:10091000C002064000030640881300200000064085
:1009200070B50024012505600623837105710379E4
:10093000002BFCD1C72A01D0042300E0012303606F
:1009400003199A710A0C641C03199A710A0A641C2F
:1009500003199A71641C02199171C1680122520431
:100960001143C160057101790029FCD100F00CFC34
:10097000002070BDF0B58FB000260D466B461E837B
:10098000090B1E82491C0391110B3446120500D03D
:100990000122891889B2099100F0AAF9000B401CC4
:1009A00081B2C4482A057DD1099B039AD2180A92C4
:1009B0008A4277D80825039804AF29460090FFF7AC
:1009C000A5FB0A000A99009801D0801A0830081A7D
:1009D0000830C008009B002A01D09B1A08338B42C4
:1009E0000ED8009B00219B1A5B199C466DE0002CE1
:1009F0006BD03B885B193B80401E491C0028F6D118
:100A00006846008A002873D003980027201A0890AF
:100A10001DD00399A848C9190A03A84905465118C9
:100A2000059100F065F9059988420CD96879FD2196
:100A300008406871687904210843687120222846BB
:100A40000599FFF76DFF08987F1CB842E1D80A9816
:100A50006946001B0390098A0027884224D0964DDE
:100A60006946098A28466118C9190A039349511829
:100A7000029100F03DF9029988420CD96879FD2174
:100A8000084068716879042108436871202228466B
:100A90000299FFF745FF6946098A03987F1C401AAF
:100AA000B84200E0C9E0DBD86846008A102505900E
:100AB00006AF29462046FFF729FB05980B4622186A
:100AC000002936D0E01A103034E0002A01D0634605
:100AD00000E0009B2C464C43E34201D12C468BE7BF
:100AE000002A02D0634601E002E0009B1C1983E764
:100AF0000998002500287DD96F4CFD2703992046D1
:100B000049190A036D49561800F0F2F8B0420BD9A2
:100B10006079384060716079042108436071202257
:100B200031462046FFF7FCFE09986D1C8542E5D34F
:100B300082E02046101A10300109002B02D0E01A82
:100B4000103000E0204690420DD80022E01A4019F3
:100B5000844676E0002E74D0388840193880491ECB
:100B6000521C0029F6D16846008B00287BD0200754
:100B700019D05148514922030546571800F0B8F8DA
:100B8000B84210D90720000387420CD36879FD21B1
:100B90000840687168790421084368715222394617
:100BA0002846FFF7BDFE6846008A201800071CD0C3
:100BB0006946098B404871180A0340490446551894
:100BC00000F096F8A84210D90720000385420CD304
:100BD0006179FD20014061716179042001436171F7
:100BE000522229462046FFF79BFE6846008B0025CF
:100BF000002800E020E01FD92F4C71190A032F496B
:100C00002046571800F074F8B84210D90F2000039E
:100C100087420CD36179FD20014061716079042124
:100C200008436071D82239462046FFF779FE6846AE
:100C3000008B10358542E0D300200FB0F0BD00E0FE
:100C400011E0002B01D0604600E020462E465643BE
:100C5000F04201D12E4682E7002B01D0604600E031
:100C6000204686197BE76846008A00260028E3D9DB
:100C7000114DA1190A0311492846571800F038F8F8
:100C8000B84210D90720000387420CD36879FD21B0
:100C90000840687168790421084368715222394616
:100CA0002846FFF73DFE6846008A08368642E0D3B4
:100CB000C2E70000FFFFFFFF0000054000F0FFFF5C
:100CC00070B50D46044600F013F8A84202D8002083
:100CD000C04370BD6079FD210840607160790421D6
:100CE00008436071202229462046FFF719FE70BD97
:100CF000124A01239178002919D1114901609F21DD
:100D00008171037101790029FCD10E4801781170BD
:100D100041785170807890700B480078C006C00E02
:100D2000022804D11078C42801D112209070907844
:100D3000834001200003181A70470000741300203C
:100D40000103000000040540A51000200E490160C9
:100D50009F2181710121017101790029FCD10B4989
:100D60000A780B4802704A78427089788170094984
:100D70000978C906C90E022904D10178C42901D114
:100D8000122181707047000001030000000405403B
:100D900074130020A510002010B50A4901604B21F2
:100DA00081710021C1710172417281720121017151
:100DB00001790029FCD1102203490448FFF73CFACD
:100DC00010BD00000510000000040540771300204E
:100DD00060300249407D087070470000A510002077
:100DE0000B2A1CD06B2A1AD0BB2A18D03B2A16D04B
:100DF000EB2A16D00423FF330133036082710A0CFF
:100E0000C2710A0A02724172FF218172C17201210C
:100E1000017101790029FCD103480078704705234E
:100E2000E9E70723E7E7000000040540F8B50446BA
:100E300001252D030698A94202D20E18AE4202D90E
:100E40000020C043F8BD6579022635436571667997
:100E500004252E4366710090204600F017F8607953
:100E6000FD21084060716079284360710020F8BD61
:100E7000F8B54579069CFD2635404571457904262F
:100E800035434571009400F001F8F8BDFFB581B01D
:100E900015460F460C460A9E0198FFF729FF874228
:100EA00002D2B919814203D90020C04305B0F0BD78
:100EB000FF2E2AD901980B2D50D06B2D4ED0BB2D73
:100EC0004CD03B2D4AD0EB2D4AD0042101221204F4
:100ED000891801608571210CC171210A0172447267
:100EE000FF218172C1720121017101790029FCD1B8
:100EF00004981E49E21B10188A15FFF79DF9FF346C
:100F0000FF3E0134013EFF2ED4D8002E23D001989D
:100F10000B2D27D06B2D25D0BB2D23D03B2D21D0E1
:100F2000EB2D21D0042132020A4302608571210C8D
:100F3000C171210A01724472FF218172C1720121C3
:100F4000017101790029FCD10498E21B10180749AE
:100F50003246FFF771F9002005B0F0BD0521B5E775
:100F60000721B3E70521DEE70721DCE700040540A0
:100F7000224A917800291AD1214901609F2181716B
:100F80000121017101790029FCD11E4801781170FD
:100F900041785170807890701B480078C006C00E70
:100FA000022804D11078C42801D1122090709278C0
:100FB0001648C721113A052A1CD213007B441B791D
:100FC000DB189F4402060B0F130042790A402832B7
:100FD00002E042790A4020324271704742790A4069
:100FE0001832F9E742790A401032F5E742790A40AF
:100FF0000832F1E742790A40EEE70000741300205E
:101000000103000000040540A51000200000054079
:10101000F7B50446FF20A071E071207260720422CF
:101020002260E36810048343E36001232371207985
:101030000028FCD1002904D0012907D002291ED0A4
:1010400099E0E06880088000E06094E0E068800853
:101050008000401CE060029800287DD0BB20A07179
:10106000FF2006302060AF20A072E06801218904D3
:101070000843E060237120790028FCD17BE0352013
:10108000FF2102312160A071012020712079002808
:10109000FCD13C4F3B78980743D40520FF21023117
:1010A0002160A0710122227120790028FCD13978B9
:1010B0001802014301204002014300202260062360
:1010C000A37122712379002BFCD1012265790323BE
:1010D000FB2635406571236023189A71401C231844
:1010E0009971090A401C20188171E0685104084375
:1010F000E060227120790028FCD1204600F044F8FD
:1011000060790421084360713520FF21023121609C
:10111000A0710120207120790028FCD13B7898072C
:10112000BBD5E06880088000801CE060E068012199
:1011300009040843E060052020607720A07140206A
:10114000A0720121217120790028FCD10298002889
:1011500011D0EB20A07100E00DE0FF2008302060EE
:10116000AF20A072E068012292041043E060217178
:1011700020790028FCD1A06940084000A06103B09C
:10118000F0BD0000000405404179C90703D0417952
:10119000490849004171C06880031BD50E483B21B6
:1011A000FF220632026081710021C1711022027299
:1011B0004172FF218172C1720122027101790029FD
:1011C000FCD106490978026004218171027101791C
:1011D0000029FCD1704700000000054000040540D4
:1011E000F8B50446C8B2091A0091FF2185180131EB
:1011F0008D4202D90020C043F8BD3B49FF27097842
:1012000085290AD00021814243D38D4241D9374AF2
:101210001E788A1816705B1C3EE0FF2A2DD8344ECB
:1012200000993B252660A5710D0CE5710D0A25720C
:101230006172A772E7720121217121790029FCD125
:10124000002A14D0D107C90F04D0284D1E784519A3
:101250002E705B1C91420AD2244F45181E78ED195E
:101260002E705E786E70891C9B1C9142F5D3812292
:1012700020480099FFF754FB11E01C4A00201D781C
:1012800081180D705D784D70801C9B1CFF28F6D96D
:1012900005E0164A8A181770491CFF29B3D90121A5
:1012A00021600620A071217120790028FCD1042042
:1012B00020606079084360710220A0710098000CE2
:1012C000E0710098000A207200986072E0680122C4
:1012D00052041043E060217120790028FCD120469F
:1012E000FFF752FF0020F8BD7413002000040540F2
:1012F0000500010000000540F0B5447985B0FD25EA
:101300002C404471447904252C43447100900C46D0
:10131000C8B2A9010E1A03929E4200D91E46201A95
:10132000E5180290E8B2B34201D9014600E000217D
:101330002F1A01910098FFF7DBFC844201D285420D
:1013400003D90020C04305B0F0BD0298874203D9FD
:10135000381A050A6D1E00E00025039F32463B4601
:1013600021460098FFF73CFFA419BE196D1E0DD34E
:10137000FF27013733463A4621460098FFF730FFF2
:10138000FF34FF36013401366D1EF3D20198002878
:1013900005D00246334621460098FFF721FF002082
:1013A00005B0F0BD10B500F001F810BD10B5082271
:1013B0000021024800F02EF810BD0000000002409D
:1013C00010B500F001F810BD10B508220121024847
:1013D00000F020F810BD00004000024010B500F001
:1013E00001F810BD10B508220221024800F012F8E1
:1013F00010BD00008000024010B500F001F810BDE3
:1014000010B502220321024800F004F810BD0000CC
:10141000C0000240F8B5002416460546002A28D927
:10142000CF000120296AA04001421FD0114B19684A
:10143000C90608D51A6810218A431A6028621A68FA
:101440000A431A6000E02862E9690B4AA240114091
:10145000AA69E1400240E2401006014338198200C7
:1014600006488258002A01D008469047641CB442BE
:10147000D7D3F8BD8001024001000100F81300201D
:1014800010B4CB0704D003689B089B001343036090
:101490008B0705D503680C24A34394002343036002
:1014A0004B0705D503683024A3431401234303608D
:1014B0000B0705D50368C024A343940123430360AD
:1014C000CB0606D5036803242402A3431402234356
:1014D00003608B0606D503680324A402A343940289
:1014E000234303604B0606D5036803242403A34368
:1014F0001403234303600B0606D503680324A403E7
:10150000A343940323430360002A03D00023032A48
:101510000AD000E001230022134303D042680904EB
:101520008A43426010BC70470122F5E702484168D7
:10153000082211434160704700000740044612A092
:1015400001F0CEFB1648216801F0CAFB154861681E
:1015500001F0C6FB1448A16801F0C2FB1348E16822
:1015600001F0BEFB1248216901F0BAFB1148616924
:1015700001F0B6FB1048A16901F0B2FB0F48E16928
:1015800001F0AEFBFEE70000496E20486172642066
:101590004661756C742048616E646C65720D0A005A
:1015A0006C5500007C5500008C5500009C550000D7
:1015B000AC550000BC550000CC550000DC550000C7
:1015C00010B500F001F810BDF8B50126B607F06AB5
:1015D0005B4CC00629D50221304600F0DFF8002818
:1015E000F9D02068017A21291FD1C18B828B491C37
:1015F0009142C28B8169895C026802D1FF31FF315F
:1016000002311161C18B491CC183C18B828B914214
:101610000BD301680A6B4B4B1A400A63036B002B18
:1016200003D0C28B81691020984720680068C16A86
:10163000490503D50121890200F086F82068006879
:10164000C16A490602D5402100F07EF82068006892
:10165000C16A49073AD5082100F0A0F8002830D027
:1016600003273F02226810680369D18C156A6D1840
:10167000491CD1842B702068017A21290FD1C28C9A
:10168000818C8A420BD2C28C521C8A4201680A6940
:1016900001D13A4302E0FF2301331A430A61C18CAE
:1016A000828C914206D1C36A002B03D0C28C016A9E
:1016B0001020984720680821006800F06FF8002883
:1016C000D0D120680421006800F03EF8206800684E
:1016D000C06A80050CD520680821006800F05EF81B
:1016E0000028F8D1206801210068490200F02CF898
:1016F00020680068C06A800620D52021304600F0AE
:1017000023F820680221006800F048F80028F8D08B
:101710002168087A002811D1CA8B8869805C306101
:10172000C88B401CC883C88B8A8B904206D30B6B36
:10173000002B03D0CA8B896910209847F8BD0000A0
:10174000AC100020EFFF0000134A1140CA0700D080
:10175000426C8A0700D5826C0A0700D5C26C8A06E3
:1017600000D5026D4A0600D5426D0A0600D5826D8D
:10177000CA0500D5C26D8A0500D5026E4A0500D59E
:10178000426E0A0500D5826E8A0401D5A82212583D
:10179000C90500D5C06D7047FF2F000081B002461B
:1017A0000092064A00201140009A7032009212689E
:1017B0000A4200D0012001B070470000FF0F7F00F7
:1017C00000220120800502600222002904D00129A4
:1017D00002D0022903D005E08168114301E081684D
:1017E0009143816081680122114381608168C9074A
:1017F000FCD1026070474268920892000A4342603E
:101800007047000030B5FFB09AB04B21C90003A863
:10181000FEF72BFD0024002500234B22D20003A954
:10182000012001F077FF9625962C2FDA002C2DDD74
:10183000601C84B2601E800003A908581021084370
:10184000611E890003AA50500022214603A8FEF71A
:1018500083FD414A07CA6B4607C30022032168463D
:10186000FEF77AFD681E800003A90858102108437E
:10187000691E890003AA50502A1BD11EE21C920047
:1018800003ABD0180022FEF767FD0EE0681E800053
:1018900003A9085810210843691E890003AA505063
:1018A0000022294603A8FEF757FD2C48C0884B218B
:1018B000C900401A82B20B4603A9012001F02AFF99
:1018C0002648C0884B21C900401A8003050C962C7D
:1018D0002FDD2046953884B2601E800003A9085889
:1018E00010210843611E890003AA5050002221469E
:1018F00003A8FEF731FD184A0C3207CA6B4607C32E
:10190000002203216846FEF727FD681E800003A918
:10191000085810210843691E890003AA50502A1B49
:10192000D11EE21C920003ABD0180022FEF714FD7A
:101930000EE0681E800003A9085810210843691EA4
:10194000890003AA50500022294603A8FEF704FD8F
:101950007FB01AB030BD000080630000F037002077
:1019600030B5002100223C4B1B689B083B4C24688F
:10197000A4081919384B1B689B08384C2468A40824
:101980001B19374C2468A4081B19364C2468A4087A
:101990001A19012806D1344B1B682024A343324C6A
:1019A000236029E002280FD12D4B1B689B08591892
:1019B0002E4B1B689B089A182B4B1B682024A343B3
:1019C0002033294C236017E0052815D1274B1B68CD
:1019D0009B089B18264C2468A4081919254B1B68E2
:1019E0009B085A18204B40335B680124E404A3434E
:1019F0001B191D4C403463601B4BC03BDB6ADB0989
:101A0000DB014C06640E2343174CC03CE3622346C3
:101A1000DB6A7F24A403A343134CC03CE362234648
:101A2000DB6A7F24E401A343D4017F25ED012C4030
:101A300023430D4CC03CE3622346DB6AAC03A34363
:101A4000054C2488A4086405AD032C402343064CB0
:101A5000C03CE36230BD0000CC120020E012002048
:101A6000BC120020C4120020C0040250D01200207A
:101A7000D8120020C812002030B500210022464BA9
:101A80001B689B08454C2468A4081919424B1B6825
:101A90009B08424C2468A4081B19414C2468A408E4
:101AA0001B19404C2468A4081B193F4C2468A40847
:101AB0001A19012806D13D4B1B682024A3433B4C37
:101AC000236039E002280FD1354B1B689B08591859
:101AD000374B1B689B089A18344B1B682024A34380
:101AE0002033324C236027E0032801D0042823D17F
:101AF0002B4B1B689B085B182A4C2468A4081919F7
:101B00002B4B1B689B089B182A4C2468A4081A19A5
:101B1000032806D1254B1B690403A343234C2361EF
:101B20000AE0042808D1214B1B6903242403A343A2
:101B300084021B191D4C23611C4BC03BDB6ADB0973
:101B4000DB014C06640E2343184CC03CE362234681
:101B5000DB6A7F24A403A343144CC03CE362234606
:101B6000DB6A7F24E401A343D4017F25ED012C40EF
:101B700023430E4CC03CE3622346DB6AAC03A34321
:101B8000054C2488A4086405AD032C402343074C6E
:101B9000C03CE36230BD0000CC120020E012002007
:101BA000BC120020C4120020C0120020C004025049
:101BB000D0120020D812002010B501F0A5FD002899
:101BC00002D0FFF71FFE06E02148006881080022CE
:101BD0002048FEF7C1FB20480068810800221F480A
:101BE000FEF7BAFBFEF7BEFB11210902884200D3C3
:101BF00010BD1B48C06A7F21890388431849C86209
:101C00000846C06A7F214905884316490988890822
:101C100049057F225205114008431149C862084610
:101C2000806AFF21490188430F4909784901FF2251
:101C30005201114008430A4988620846806B000A35
:101C400000020A49097808430549886300BFCFE7C5
:101C5000B8120020A45B000060610000805B0000FF
:101C600000040250CC1200207A610000786100006C
:101C700000B50C48806A1F2149038843012189036C
:101C80004018084988620846806A0C218843054943
:101C9000886205480068810800220448FEF75CFB62
:101CA00000BD0000000402506C6100009C5B00005D
:101CB000F0B587B005460027EB480690EB48059045
:101CC0000020049003900026092D05DD2720C04345
:101CD000854201DA07B0F0BD2846283045B201F050
:101CE00013FD002808D00A20684383B20A226946FF
:101CF000002001F00FFD07E00A206843DC4A81184C
:101D00000A226846FEF798FA6846808880010490A7
:101D1000D8488068D849084004990843D549886064
:101D20006846C078C0000390D44800687821884392
:101D300003990843D14908606846807900040699F0
:101D4000084306900022012106A8FEF705FB68461D
:101D5000C07900050599084305900022012105A8D6
:101D6000FEF7FAFA002019E08100C54A1268515ABC
:101D70000904090E7A2910D18100C14A126851580C
:101D80000722520591436A461278520511430F46C5
:101D90008100BB4A1268575005E0401CB9490968E8
:101DA00089088142E0D800BF002019E08100B64ACE
:101DB0001268515A0904090E7A2910D18100B24AD9
:101DC000126851580722520591436A46127852050B
:101DD00011430F468100AC4A1268575005E0401C81
:101DE000AA49096889088142E0D800BF002019E0AB
:101DF0008100A74A1268515A0904090E7A2910D1A4
:101E00008100A34A126851580722520591436A463D
:101E10001278520511430F4681009D4A12685750AF
:101E200005E0401C9B49096889088142E0D800BF51
:101E3000002019E08100984A1268515A0904090EDD
:101E40007A2910D18100944A12685158072252050C
:101E500091436A461278520511430F4681008E4A1B
:101E60001268575005E0401C8C4909688908814276
:101E7000E0D800BF002019E08100894A1268515A59
:101E80000904090E7A2910D18100854A1268515837
:101E90000722520591436A461278520511430F46B4
:101EA00081007F4A1268575005E0401C7D4909684F
:101EB00089088142E0D800BF684681784078800078
:101EC00008436946097A490108430446002017E09F
:101ED00081006B4A1268515A0904090E70290ED10B
:101EE0008100674A12685158ED221204914322047E
:101EF00011430E468100624A1268565005E0401CAC
:101F00006049096889088142E2D800BF002017E0D3
:101F100081005D4A1268515A0904090E70290ED1D8
:101F20008100594A12685158ED221204914322044B
:101F300011430E468100544A1268565005E0401C79
:101F40005249096889088142E2D800BF002017E0A1
:101F500081004F4A1268515A0904090E70290ED1A6
:101F600081004B4A12685158ED2212049143220419
:101F700011430E468100464A1268565005E0401C47
:101F80004449096889088142E2D800BF002017E06F
:101F90008100414A1268515A0904090E70290ED174
:101FA00081003D4A12685158ED22120491432204E7
:101FB00011430E468100384A1268565005E0401C15
:101FC0003649096889088142E2D800BF002017E03D
:101FD0008100334A1268515A0904090E70290ED142
:101FE00081002F4A12685158ED22120491432204B5
:101FF00011430E4681002A4A1268565005E0401CE3
:102000002849096889088142E2D800BF684681787A
:102010004078800008436946097A4901084304462C
:10202000002017E08100204A1268515A0904090E65
:1020300070290ED181001C4A12685158ED221204F9
:102040009143220411430E468100174A12685650EC
:1020500005E0401C1549096889088142E2D800BFA3
:10206000FEF780F900BF35E612570000124E20003F
:102070008A610000400003403F00FFFF400007402E
:10208000F0120020BC120020F8120020C012002024
:10209000F4120020C4120020FC120020C8120020FC
:1020A00020130020EC12002010130020CC1200207E
:1020B000012906D1C0221258CB021A43C0231A505C
:1020C00006E0C02212580123DB029A43C0231A50B3
:1020D000704710B5C022125818239A43CB00182419
:1020E00023401A43C0231A5010BD012906D1C02233
:1020F00012588B021A43C0231A5006E0C02212580D
:1021000001239B029A43C0231A50704702460029BC
:1021100004D1DC208058C007C00F7047DC208058F5
:1021200001231B041840000CF7E7012906D1C02247
:1021300012580B021A43C0231A5006E0C02212584C
:10214000FF2301339A43C0231A50704710B5C022B1
:10215000125803231B039A430B0303242403234035
:102160001A43C0231A5010BDF7B583B0134600219F
:1021700010CB01941C68029400BF64E001248C40E1
:10218000049D2C40002C5CD00C4601250095009D40
:10219000002D0BD0FF2501352D5826461836012776
:1021A000B7403D43FF26013635500AE0FF25013593
:1021B0002D58264618360127B740BD43FF26013665
:1021C000355000BF00290FD1CC242458019D2C4646
:1021D000CC252C50D0242458240A2402029DEDB290
:1021E0002C43D0252C502CE04C1EA6000446E03495
:1021F000019DA551042911DCFC2422584C1EE50048
:10220000FF24AC401546A5432A46029CE4B24D1E6D
:10221000ED00AC402243FC24225012E0FF240134A4
:1022200022584C1FE500FF24AC401546A5432A4622
:10223000029CE4B24D1FED00AC402243FF24013468
:1022400022504C1CE1B2082998DB06B0F0BD30B535
:10225000FF2305331B5802242343FF240534235056
:1022600000290DD123461B5803246403A3435403C0
:1022700003256D032C402343FF24053423500DE038
:10228000FF2305331B580324E403A343D40303258E
:10229000ED032C402343FF240534235030BD002997
:1022A00010DDC82212580123DB031A43C8231A5039
:1022B000C822125892B20B041B0C1B041A43C823E9
:1022C0001A5006E0C82212580123DB039A43C823A0
:1022D0001A507047F8B504460E4617461D46002EA4
:1022E0000FD1D420005929680846D42108512D1D4A
:1022F000D8200059000A000229780843D821085143
:102300001BE0012E05D12A4639462046FFF72CFF57
:1023100013E02A4639462046FFF726FFD42000590D
:1023200029680846D42108512D1DD8200059000ADB
:10233000000229780843D8210851F8BD30B500299A
:102340000AD1C0231B581B021B0A1406240E2406A4
:102350002343C02423500BE0C0231B58FF24240434
:10236000A3431404FF252D042C402343C0242350F1
:1023700030BD000030B500290BD1DC231B580B4CBD
:1023800023405400094DED432C402343DC242350CB
:102390000AE0DC231B58064C23405404044DED4353
:1023A0002C402343DC24235030BD000001F0FFFF0C
:1023B000FFFF01F05621095C2030CA060749D20E02
:1023C0000A7002781207120FCA70027E5206520F6C
:1023D0004A7000790007000F88707047A71000202E
:1023E00010B500F001F810BD10B5024800F010F86B
:1023F00010BD0000B010002010B500F001F810BDB5
:1024000010B5024800F004F810BD0000E4100020F0
:1024100010B501680446C8690122C007C00F002832
:1024200003D0086A1043086210BDC8690422104234
:1024300026D0C868400723D520688168608B626910
:102440004300D218401C60831180618B208B814235
:1024500012D3236A2046002B03D0428B10206169DF
:102460009847216804224869904348612268022104
:1024700050698843506103E02068C0684007DBD49E
:1024800021680222C869104226D0C868400723D5B7
:1024900020688168608B62694300D218401C6083A9
:1024A0001180618B208B814212D3236A2046002B3E
:1024B00003D0428B1020616998472068042142694B
:1024C0008A4342612168022248699043486103E0DF
:1024D0002068C0684007DBD420680821C2690A422E
:1024E000A2D0C068800737D5608A218A884217D277
:1024F000608A2168E2684300D218401C608210881C
:1025000088602068C16849070AD5A17A112907D1D6
:102510008168608B62694300D218401C608311801F
:10252000618A208A814213D32079002803D1206850
:10253000C168C906FCD4636A002B03D0628A1020EC
:10254000E16898472268082150698843506103E098
:102550002068C0688007C7D4A07A012800D063E74C
:102560002068C1684907FAD58168C1684907FBD46A
:1025700010BD401E0AD300BF00BF00BF00BF00BF98
:1025800000BF00BF00BF00BF401EF4D27047000074
:102590000349CA6F9207D217521CFAD108607047DC
:1025A0000030004010B5104841690904090F0ED0F1
:1025B000491C42690D4C920510D5806A04221040D6
:1025C000042806D00A48FDF7A1FD606010BD012176
:1025D000EFE70848FDF79AFD606010BD0648FDF77B
:1025E00095FD606010BD0000000004409C100020BC
:1025F000006CDC020090D0030048E801F8B5054605
:10260000FF2701372B463B220021A5480097FEF704
:102610000DFC2846AA7F1E30002113462E24467842
:10262000B2188678801C7118D2B2C9B2641EF6D175
:10263000501829466031CA7EC0B282427ED1C87D20
:10264000022812D32031087800223F244E78301817
:102650008E78891CB218C0B2D2B2641EF6D1FF21A6
:102660008018495DC0B2814275D18E49086A8E4A90
:102670002C4610405A07920E10432034A27A52067C
:10268000520F120410430862486A884A10402278A8
:102690001207520E1043A2795207520A10434862A1
:1026A000886A834A104022791207D20E1043A2781A
:1026B0001207D20A10438862C86A237A78221B075D
:1026C00090435B0E1843C8627A480368267A9343A6
:1026D0003609F600334303600B6B667A9343360783
:1026E000760E33430B63CB6B667A93433609F60061
:1026F0003343CB6341689143A27A1207520E1143D0
:102700004160C168E27AC908C9005207520F1143FB
:10271000C160694FF969FF2212029143E27C120203
:102720001143F961B969654A1140227E1207120E00
:102730001143627E12021143B96100E00BE02A46A8
:102740004032117DCE064B09F60E5B01361D1F2E61
:102750000AD91F2109E05A49002008703946284645
:10276000FDF783FD0020F8BD091DC906C90E0B4306
:102770001375016901235B059943937DDB079B0A70
:102780001943016147498B6B4E4E3340967DF606E7
:10279000360FB6003343167D527DF606B60CD206D0
:1027A0003343520B13438B63826813022A46603211
:1027B00016791B0A360633438360D37D022B1FD361
:1027C000042B08D2237E0726F341012676079B19A6
:1027D0001926F34123768B6A07267605B343267EB6
:1027E0007606760F760533438B62066901231B0656
:1027F0001E430661D07D072802D3886A1843886289
:10280000D07D062836D3086A06229043227C92099E
:10281000520010430862386A70218843A17B49073F
:10282000490E08433862786A012189028843A17BF6
:102830000907C90F890208437862F8693021884383
:10284000A17B8906890F09010843F861B96A1E480E
:102850000140E07B4206920F12011143C206920F23
:10286000920140071143400D0143A07B8009C00243
:102870000143B9622846FDF7AFFD2846FFF79AFDF0
:102880002846FEF7A5FA064C2046FEF785FA2046B4
:10289000FEF75CFA2046FEF76BFB0120F8BD000056
:1028A0000000054000000740C7FFF8FF87FF8FFFCB
:1028B000E1FFE1FF40000740000004400F00FFFF80
:1028C0009C100020C301F8FF0FE0FFFF70B5174810
:1028D0000025C561164CE06A0F2109048843E062B7
:1028E000144E2A4601213046FEF792FB0121304664
:1028F000FEF766FFFDF70AFF0F480561606A3F219A
:102900000901884360620D48416B490849004163F1
:102910000B490A6810239A430A60016A0622114390
:102920000162206A70210843206270BD40000740A8
:10293000000004400000054000000840000007407F
:102940008001024070B50446006881680125C9070E
:10295000002903D08560E16A0120884720688169E9
:10296000C907C90F03D08561E16A02208847216841
:10297000104A0E2302268868914201D1184000E0D7
:102980003040002814D08868914201D1184000E0FE
:102990003040886020688168904201D1702200E058
:1029A00004221140816020688560E16A0320884725
:1029B00070BD00000080004010B500F001F810BDAF
:1029C00010B50248FFF7BEFF10BD0000181100202F
:1029D00010B500F001F810BD10B50248FFF7B2FFC6
:1029E00010BD00004811002010B500F001F810BD26
:1029F00010B50248FFF7A6FF10BD000078110020B7
:102A0000002904D00269120E12060A4302617047BF
:102A100010B500F001F810BD10B5024800F010F834
:102A200010BD0000A811002010B500F001F810BD85
:102A300010B5024800F004F810BD0000DC110020C1
:102A400070B501688A68130702461B0F2032042BF9
:102A500037D00CDC012B11D0022B0FD1137A002BB5
:102A60000CD0C96F8907C917491C2CD03DE0062B33
:102A700005D00C2B02D10C2100F049F870BD0446A2
:102A80004869C505507AED0D0028F7D06669002E1B
:102A9000F4D0680704D5E38C04212046226AB047AD
:102AA000280705D5E38C666905212046226AB047D0
:102AB000A807E3D5E38C656906212046226AA8476A
:102AC00070BD0421D8E7C38B818B8B420DD2C18BA3
:102AD000036884696418491CC183217819600168FE
:102AE000C96F8907C917491CEDD0C18B838B9942E7
:102AF000E6D101684B680224A3434B6000211172A8
:102B00004469002CDCD0C38B8269A04770BD70B5CE
:102B100004462030427A002A56D0257C0022042325
:102B2000002D52D00C290BD112E0E18CA28C9142E5
:102B30003ED20168E08C226A1218401CE0841170B9
:102B4000206884210958C906C90E0129EDD82FE053
:102B50002168C96F0907C917491C11D1E18CA58CDF
:102B6000A9420DD221680D68E18C266A7618491CAD
:102B7000E18435702168C96F0907C917491CEDD078
:102B80002168CD6F2D07ED176D1C11D04D686D08B4
:102B90006D004D6021684D689D434D604272227406
:102BA0006569002D04D0E38C02212046226AA847E3
:102BB000E08CA18C884207D36569002D04D0E38C9A
:102BC00003212046226AA84770BD2168C96F090702
:102BD000C917491C11D1E18CA58CA9420DD22168DD
:102BE0000D68E18C266A7618491CE18435702168ED
:102BF000C96F0907C917491CEDD0E18CA58CA94202
:102C0000E2D121684D686D086D004D6021684D6806
:102C10009D434D6042726569002DD5D0E38C012142
:102C20002046226AA84770BDF8B50D460446FDF758
:102C300083FCE268002180263243E2602A680B466A
:102C400097001922FDF7A8FA3A460023FDF774FA17
:102C50000746642801D20020F8BD6421FDF756FA2A
:102C6000C1B221600104090E616064214843381A31
:102C700000013230FDF74AFAC0210851E068B04344
:102C8000E060E0688109287989010843E06001205B
:102C9000F8BD10B500F002F810BD0000054801684D
:102CA00008221143016004480068002800D0004752
:102CB00070470000006000401012002010B500F0C6
:102CC00001F810BD0449012088600448006800280C
:102CD00000D0004770470000007000401412002030
:102CE0000FB410B503A9044B044A029800F030F861
:102CF00010BC08BC04B01847FD360000301300209B
:102D0000F0B4040C8BB2264682B25E430D0C104622
:102D1000370C5843360480190021794116466E431A
:102D2000370C36048019794126466E438919F0BC68
:102D3000704702E008C8121F08C1002AFAD1704784
:102D40007047002001E001C1121F002AFBD170472B
:102D5000FFB591B00F460546002606E025280AD0AB
:102D6000149A139990476D1C761C28780028F5D189
:102D7000304615B0F0BD002400940121F34A0294BE
:102D800000E004436D1C2B780846203B984010421D
:102D9000F7D128782A280ED0022128780246303A26
:102DA000092A15D8009A0A235A43303A80180C434E
:102DB0006D1C0090F1E701CF0090002805DA01209A
:102DC00040030443009840420090022004436D1CDD
:102DD00028782E2815D10420044368786D1C2A28F1
:102DE0000AD101CF6D1C02900BE002990A225143D7
:102DF000303940186D1C0290287801463039092975
:102E0000F3D928786C2810D006DC4C281AD0682812
:102E10000ED06A2817D104E0742813D07A2812D172
:102E200010E00120400504430CE00121090501E008
:102E3000032109050C436978814203D10120000573
:102E400024186D1C6D1C287803906E281ED00CDC95
:102E5000632831D004DC00288AD0582811D1B2E090
:102E600064287BD069280CD178E073282DD004DC4D
:102E70006F2870D0702804D1A7E075286CD078280E
:102E80006BD0149A13999047761C62E06002400F51
:102E9000022807D003280AD0042838680AD0066020
:102EA0003F1D56E03868F11706604160F8E7386862
:102EB0000680F5E70670F3E7387869460874002065
:102EC000487404A80390012003E0386803900020B0
:102ED000C0433F1D61070FD5002101E00199491C46
:102EE000029A0191914213DA8142F7DB019A039928
:102EF000895C0029F2D10BE0002101E00199491C15
:102F000001918142FADB019A0399895C0029F5D18C
:102F100001990098139A401A00902146149B00F0E2
:102F20003BF901998019461807E003980399007846
:102F3000491C0391149A139990470198401E0190DF
:102F4000401CF2D12146149B139A009800F014F90A
:102F500086196D1C09E741E033E034E00A200021C6
:102F6000049005916002410F022905D001CFC217DC
:102F70009446032905D007E0FF1DFF08FF0003CF9B
:102F800006E000B2C2179446042902D140B2C1172C
:102F90008C4600226146944506DA0A4600214042EA
:102FA00091418C462D2102E0210504D52B216A4652
:102FB0001176012103E0E10701D02021F7E701911B
:102FC00054E00A200BE0102009E0102004900021BA
:102FD0000420044308200591029003E0082000210A
:102FE000059104906002410F022905D001CF002213
:102FF0009446032906D006E0FF1DFF08FF0003CF1B
:103000008C4603E080B2042900D1C0B200210191B6
:1030100021072BD50399702906D0049A1021059B0E
:103020004A401A4305D00EE040216A46117601213C
:1030300008E06146014306D030216A4611760399C3
:10304000517602210191049A0821059B4A401A43B6
:103050000CD16146014301D1610707D530216A4691
:103060001176012101910299491E02910399582973
:1030700004D037A103910FA90F910DE039A1F9E711
:103080006146059B049AFDF757F8039B8C469B5CB1
:103090000F9A521E0F92137061460143F0D10F98A0
:1030A00007A9081A20300390600704D50120000406
:1030B0008443029801E0012002900399884201DDD7
:1030C000401A00E000204118029001980918009869
:1030D000401A0090E00306D42146149B139A0098EE
:1030E00000F05AF886190020049008E006A9085C50
:1030F000149A139990470498401C761C04900199E7
:103100008842F3DBE0030CD52146149B139A009808
:1031100000F042F8861904E0149A30201399904781
:10312000761C0299481E02900029F5DC08E00F98F1
:103130000F990078491C0F91149A13999047761CA7
:103140000399481E03900029F1DCFBE609280100E1
:10315000303132333435363738396162636465660D
:1031600000000000303132333435363738394142CF
:103170004344454600000000F8B5044600251E46BD
:103180001746880404D405E039462020B0476D1C5A
:10319000641EF9D52846F8BDFFB50446002581B068
:1031A0001E46C80301D5302700E02027880404D537
:1031B00005E038460399B0476D1C641EF9D52846D2
:1031C00005B0F0BD3EB50446304800900022012114
:1031D0006846FDF7C1F82E48009002AA0121684612
:1031E000FDF7BAF82B48009001AA01216846FDF7C7
:1031F000B3F822460199029800F05AF8002800D14D
:103200003EBD2548009002AA01216846FDF7A4F8BA
:103210002248009001AA01216846FDF79DF8224648
:103220000199029800F044F8002800D1E8E71C4812
:10323000009002AA01216846FDF78EF81948009017
:1032400001AA01216846FDF787F8224601990298F4
:1032500000F02EF8002800D1D2E71348009002AA0F
:1032600001216846FDF778F81048009001AA012175
:103270006846FDF771F822460199029800F018F8A7
:10328000002800D1BCE70120BAE7000012FF0100CE
:103290001361000013620000136300001364000058
:1032A0001371000013720000137300001374000008
:1032B0000346002B06D0FF20401A401C904205D93F
:1032C00000207047914201D90020FAE70120F8E779
:1032D00070B5FFB085B00026002002900024812048
:1032E000800003AB0B220121890200902B48FDF7DF
:1032F0009DFDFF34FF3402342949684680890880E7
:1033000028496846C08908800846008826498842BE
:1033100003DC24480088002803D100207FB005B0DA
:1033200070BD15E032460121490203A802F05EF9A2
:10333000064681208000009001208002211803AB06
:103340000B221648FDF772FDE01DFF30FA3084B203
:1033500014480088001D8442E4DB12480088001DE8
:10336000201A01214902081A85B23246294603A8CB
:1033700002F03CF9064603A84119042202A8FCF712
:103380005BFF0298B04206D101200849087002F0A4
:1033900087F90120C2E70020C0E7000000000540D7
:1033A0002613002028130020FC0B00002A13002005
:1033B000F8B5154C0746A06B02263043A063A06BFE
:1033C00004218843A063114D39462846FFF718FBB6
:1033D000296801200909090101432960E9680420DD
:1033E0000142FBD0E9680143E960AD69384608490C
:1033F000FFF786FC2A460023FCF79EFE054908607D
:10340000A16BB143A163F8BD00000440006001401E
:103410000048E8012812002010B50E4982B0086863
:1034200049680191009001210820FDF779F80A48C8
:1034300041680A4A114040314160094C69462046C2
:10344000FFF7F2FBE06901210843E061E069A06059
:1034500002B010BDA858000000000340BFBFBFFF6E
:103460000030004010B5FCF783FF10BD014900207B
:10347000487070475812002010B5FCF779FF10BD56
:10348000F0B50646FFB084B0012040020024009051
:10349000254602AB3B2231462D48FDF7E9FC37219A
:1034A0000598090388424ED80146FF200130814229
:1034B00049D9FF36FF36023600293DD9EF1D059860
:1034C000F937B84215D3FF20013000907119214B14
:1034D0003B221F48FDF7CCFC1F4800223D468021BF
:1034E00043781C198378801C9A18491EF8D1A418B7
:1034F0001FE0401B00907119164B3B221448FDF74A
:10350000B7FC05991348491B0904090C10D0401E4B
:10351000CA0702D042781419401C0022490806D07C
:1035200043781C198378801C9A18491EF8D1A41876
:10353000059D0598A842C1D80A98A04203D17FB042
:10354000012004B0F0BD7FB0002004B0F0BD000049
:1035500000000540601400205F14002010B50146F3
:103560000148FDF7ADFB10BD00000540F0B5FFB010
:103570000F46054684B005214748490301600126EE
:1035800076020024294602AB3B2244480096FDF710
:103590006FFC02A80190404800960168BE198E4257
:1035A0000FD839463D48009B019AFDF7A5FE0598C6
:1035B000FF352830FF3502353746059000280DD8F5
:1035C00055E03648FDF77CFB002800D0FEE7324985
:1035D00001200A68000310180860E2E7E61DF936CA
:1035E000B04228D3FF200130009029192C4B3B22F8
:1035F0002A48FDF73DFC2A480190FF2001303C1984
:1036000022180090244801688A4207D8214623489E
:10361000009B019AFDF770FE344625E01F48FDF738
:103620004FFB002800D0FEE71B4801210268090378
:1036300051180160EAE7001B00902919184B3B2242
:103640001648FDF715FC1648009005983E19041B16
:103650001148321901688A4210D8234631460F4872
:10366000009AFDF749FE059C0598A042B6D8294668
:103670000A48FDF725FB7FB004B0F0BD0748FDF711
:103680001FFB002800D0FEE7034901200A68000361
:1036900010180860E1E70000541200200000054007
:1036A00060140020052002494003086070470000B4
:1036B00054120020F7B50F4C1546064642192168F2
:1036C0000D488A4203D82B463146019A0EE0074640
:1036D000FDF7F6FA002800D0FEE701212068090373
:1036E000401820602B4631463846019AFDF704FE0B
:1036F00003B0F0BD541200200000054010B5044690
:10370000FEF746FF204610BD0148007870470000D4
:103710002A130020FFB581B004460F461646A000CC
:103720001F49401840881F49884205DCA0001C49F9
:1037300040184088002802D1002005B0F0BD002EBE
:1037400013D0A000164A0096105A01229202801847
:10375000C01C049A81183B460B221348FDF766FBF8
:103760000546002D1AD13046E7E7A0000C49401865
:1037700040880090A0000A46105A01229202801848
:10378000C11C3B460B220848FDF750FB0546002DA7
:1037900004D1A000024940184088CEE70020CCE7C1
:1037A000F0370020FC0B0000000005400249496989
:1037B000491C0160704700000000025070B531A044
:1037C000FFF78EFA344A3549002001F08FFE344A63
:1037D0003449012001F08AFE334A3449022001F0C5
:1037E00085FE334A3349032001F080FE01F086FE56
:1037F00031A133A0FFF774FA32A0FFF771FA2EA1BE
:103800002FA0FFF76DFA0521490339A0FFF768FAE9
:1038100029A12BA0FFF764FA372109033DA0FFF788
:103820005FFA25A126A0FFF75BFA0121490242A019
:10383000FFF756FA4948FCF7A1FD72B601F0B6FD54
:10384000FF214748CD3141600025456045498160F1
:1038500085604549681E086044490860444C3B2225
:1038600029462046FDF7BCFA01208005056051205D
:10387000400201684268606181F308889047002037
:1038800070BD00000A426F6F746C6F6164657220D6
:10389000696E2E2E0A0A000075390000555300008B
:1038A000653A0000F55300006D3B000041540000F4
:1038B000E13900008D5400005B495D2000000000EC
:1038C00025730000436C65616E20757020616E6425
:1038D0002074727920746F206A756D7020696E741F
:1038E0006F2061707020696D6167652E2E0A00007F
:1038F0002D2061707020706172746974696F6E2020
:10390000737461727420616464723A20307825782F
:103910000A0000002D20617070207061727469745B
:10392000696F6E2073697A652020202020203A205C
:10393000307825780A0000002D2061707020696DB4
:10394000616765206865616465722073697A6520C6
:1039500020203A20307825780A0A0000102700003D
:1039600000000440FF7F010080E100E080E200E011
:103970000000054010B507A108A0FFF7B1F908A0A5
:10398000FFF7AEF90521412049030003FFF7EEFDE3
:1039900010BD00005B495D200000000025730000A1
:1039A00054727920746F206D6F766520696D616740
:1039B000652066726F6D20417070204261636B7587
:1039C0007020506172746974696F6E20746F204149
:1039D000707020506172746974696F6E2E2E0A00C7
:1039E00070B50CA10DA0FFF77BF90DA0FFF778F9DA
:1039F0001A4DE87808280CD0194C002628780028A1
:103A000004D02E702178201D00F012FFE8780828DD
:103A1000F4D170BD5B495D200000000025730000FB
:103A2000456E746572696E6720507269766174655F
:103A300020322E3447202850524629204F5441200E
:103A4000666C6F772C204F544120536572766572F7
:103A500020496E69742E2E0A0000000058120020C2
:103A60009015002084B02FA130A0FFF739F930A0C5
:103A7000FFF736F93548FCF781FCFFF713FE01210B
:103A80000820FCF741FD01210820FCF749FD3048E2
:103A90004168304A11404031416041682E4A11402E
:103AA000803141602D484168420491434160E120EA
:103AB0000003009003206946294C08712046FFF757
:103AC000B3F8E06901210843E061E069A060E169C1
:103AD00002200143E161E169A160E1698143E161A3
:103AE00020682715052676031E4C5925029030467E
:103AF000FCF74AFCB84211DD3046FFF7C1FC002854
:103B000002D13046FFF72AFD16218820256021606A
:103B100020602268002AF9D0FCF7AEFD1248FEF7BB
:103B200028FDE4E75B495D200000000025730000EC
:103B3000456E746572696E67205541525420444643
:103B40005520666C6F772E2E0A00000010270000AB
:103B500000000340BFBFBFFF7F7F7FFF40000240E8
:103B6000003000404000034040420F0010B50FA15C
:103B700010A0FFF7B5F810A0FFF7B2F81548FCF752
:103B8000FDFB5920144C1622882120602260216000
:103B90002368002BF9D0FCF777FD00BF00BF00BF02
:103BA00000BF00BF0020206010BD00005B495D2009
:103BB0000000000025730000456E746572696E6731
:103BC000205553422044465520666C6F772E2E0AAE
:103BD000000000001027000040000340F0B5C7B00F
:103BE00063A0FFF77DF806A8FEF708FD694E0028E0
:103BF0002DD069A0FFF774F820A8417B68A0FFF7DB
:103C00006FF820A8817B6DA0FFF76AF820A8C17B20
:103C100071A0FFF765F820A8C07B02281BD320A85D
:103C2000008B308120A8408B708120A8808BB081D0
:103C300020A8427F017FC07E00900292019120A8BF
:103C4000837E427E017E6BA0FFF74AF81BE075A0E1
:103C5000FFF746F82AE010A8C08F308120A800881E
:103C6000708120A84088B08120A8C27881784078EF
:103C700000900292019120A8037818A8C27F817F4A
:103C80005CA0FFF72DF820A8037BC27A817A407AE6
:103C900002AC0FC420A8017AC0790090019120A83D
:103CA0008379427901796EA0FFF71AF87BA0FFF7BC
:103CB00017F8804D00242819C1787FA0FFF710F86D
:103CC000641C102CF7D3A978012528468840810A66
:103CD0007BA0FFF705F8824C616A20462F04394328
:103CE000616280490A6904239A430A610021FDF751
:103CF00082FD7D488169294381618169C901FCD5C3
:103D0000054640690121890288436861606849026B
:103D1000884360606068490008436060FA20FEF7ED
:103D200028FC286A40084000286228687060A06962
:103D3000306060680821084360606C48C1680222F6
:103D40001143C1600020A060E0602061A069384399
:103D5000A06167491007086066490868FF221202DF
:103D60009043032292031043086047B0F0BD000067
:103D700054727920746F206C6F61642048572063FF
:103D8000616C6962726174696F6E20646174612E26
:103D90002E0000001812002020444F4E452E0A002D
:103DA0002D204368697020496E666F2020202020F6
:103DB000202020203A20307825780A002D204368E2
:103DC00069702043502056657273696F6E20202001
:103DD0003A2025640A0000002D20436869702046BF
:103DE000542056657273696F6E2020203A20256436
:103DF0000A0000002D2043686970204D4143204196
:103E000064647265737320203A202530325825305F
:103E10003258253032582530325825303258253026
:103E200032580A000A5741524E494E473A204361E0
:103E30006E6E6F742066696E642076616C696420B2
:103E400063616C6962206461746120696E206375CE
:103E50007272656E742063686970210A0000000048
:103E60002D204368697020554944202020202020BF
:103E7000202020203A202530325825303258253055
:103E800032582530325825303258253032582530B6
:103E9000325825303258253032580A002D204368D8
:103EA000697020466C6173682055494420202020A9
:103EB0003A20000074130020253032580000000022
:103EC0000A2D204368697020466C6173682053692D
:103ED0007A652020203A20256C64204B420A00009D
:103EE0000000074000ED00E0000004400000025028
:103EF00000E100E01CE400E000B587B018220949A9
:103F000001A8FCF799F90022062101A8FCF724FA80
:103F10000548406801214904884340180249486027
:103F200007B000BDE45A00000005025000284BD144
:103F30004B4A126901239B039A43D218484B1A61DA
:103F4000012906D11A461269CB039A43D218444B71
:103F50001A61434A526801235B059A43404B5A60F9
:103F60001A46126801239B029A43D2183C4B1A60EE
:103F70001A46126801239B039A43D218384B1A60E1
:103F80001A461268FF2301339A43D218344B1A6041
:103F90001A4692697F231B029A4353231B02D218AD
:103FA0002F4B9A611A4612680123DB039A43D218F9
:103FB0002B4B1A602A4A4032526852085200521C57
:103FC000274B40335A604AE0254A12690123DB033C
:103FD0009A43D218224B1A61012906D11A46126956
:103FE0008B039A43D2181E4B1A611D4A5268012353
:103FF0005B059A431A4B5A601A46126801239B02CA
:104000009A43D218164B1A601A46126801239B0372
:104010009A43D218124B1A601A461268FF230133D2
:104020009A43D2180E4B1A601A4692697F231B02DC
:104030009A4353231B02D218094B9A611A461268FD
:104040000123DB039A43D218054B1A60044A40321D
:10405000526852085200521C014B40335A6070475C
:10406000C004025030B5A3B00025FFF74DFB002877
:1040700006D000231A4622A90E20FFF74BFB07E0CB
:104080002748017820A801722548417820A841726C
:104090008422244901A8FCF7CFF820A9087AFFF769
:1040A00091F8002803D00125012023B030BD002461
:1040B00014E0A0001C494018006802900022212151
:1040C00001A8FCF749F920A9087AFFF77BF8002836
:1040D00002D001250120E8E7601CC4B2052CE8D31A
:1040E000002D18D1002414E0A0000F4940180068EA
:1040F00002900022212101A8FCF72EF920A9487A7C
:10410000FFF760F8002802D001250120CDE7601CF0
:10411000C4B2052CE8D301F0D1F82846C5E7000069
:1041200088610000FC5A0000C45A000000B5024833
:10413000FFF73CFB00BD0000AC1200201CB504469C
:10414000204600F02BFACE4840680121490508437B
:10415000CB494860CA4840304068012109050843FE
:10416000C74940314860E07B801EC1B2C448C038B6
:10417000FDF7ECFFE27B214610316846FCF75CF866
:10418000627E6B460221BE48C038FEF7A3F8E07B92
:10419000022801D1FFF7B0FE2079002805D10021C7
:1041A000B748C038FDF7A1FF1DE00121B448C03871
:1041B000FDF79BFF2079032807D1B1480068012152
:1041C00089030843AE4908600DE0AD48006801214D
:1041D000490288432179491E4902012252021140B5
:1041E0000843A74908606078032808D1607B01284C
:1041F00005D00021A248C038FDF797FF0CE0A04889
:104200000068FF210131884361790902FF220132F0
:10421000114008439A490860607B012817D100BF0C
:10422000002808D096494039096C80221143944AED
:10423000403A116407E092494039096C8022914369
:104240008F4A403A116400BF012000F055FD607BA9
:10425000022859D100200EE081008A4A1268515A82
:104260000904090E7E2905D187498200854B1B6808
:10427000995005E0401C8549096889088142EBD8BE
:1042800000BFFCF76FF87E484030406820210843AB
:104290007B494031486008464068012109060843CF
:1042A000774940314860084640680121C902084307
:1042B00073494031486008464068012109030843BA
:1042C0006F494031486008464068FF21C13188434A
:1042D0006B4940314860084640688021084368497E
:1042E0004031486066480069FF2101310843644954
:1042F000086108460069032149028843FF30FF3006
:1043000002305F4908610CE06078032809D15C48FD
:1043100040304068012149068843401858494031DF
:1043200048602079002811D0554800680121C90350
:104330008843E17D002901D1012100E00021C9036A
:104340000122D203114008434D49086060790128D9
:1043500010D14B484030406840084000217E002981
:1043600001D1012100E00021C907C90F08434449D8
:10437000403148602078002805D100214048C038ED
:10438000FDF796FE04E001213D48C038FDF790FEA0
:10439000A27B01213A48C038FDF7D0FF20780028E1
:1043A00007D1607B022804D101213548C038FDF7D0
:1043B0007FFEA07D002803D00021204600F028FACF
:1043C000002033490870E07800F024FC20780228AF
:1043D00014D12B48006840218843294908600846C9
:1043E0000069FF21013188432549086108460069B9
:1043F0000121C9020843224908610AE020480068F7
:1044000040218843217889014022114008431C49FA
:104410000860E078032802D0E078042803D12178EE
:10442000A078FFF783FD204600F008FC14480068E0
:1044300002218843217B4900022211400843104990
:10444000086021890E48C038FDF729FF1148002176
:1044500002680B48C038FDF78DFF0F4800688208DE
:1044600001210748C038FDF785FF0548006840086E
:104470004000A178C907C90F0843014908601CBD65
:10448000C0040250FC120020027E2601C812002047
:10449000AA1200202C1200203412002004480168C7
:1044A0000902090A016001200249C0020860704740
:1044B00008E400E000E100E0054804490160054926
:1044C0008160054941600549C16070477934000049
:1044D000D4370020650A00206D34000065340000E8
:1044E00010B58CB00446012C0AD11422274907A824
:1044F000FBF7A2FE0022052107A8FBF72DFF42E0F3
:10450000022C0BD120222149143104A8FBF794FE80
:104510000022082104A8FBF71FFF34E0032C24D15C
:1045200028221A49343102A8FBF786FE00220A210C
:1045300002A8FBF711FF00200EE08100144A126868
:10454000515A0904090E7F2905D112498200104BE6
:104550001B68995005E0401C0F4909688908814291
:10456000EBD800BFFBF7FEFE0DE0042C0BD12C2294
:1045700006495C3101A8FBF75FFE00220B2101A870
:10458000FBF7EAFE00BF0CB010BD0000B8630000EE
:1045900010130020027FC120CC12002070B5054608
:1045A00001461A222048FBF747FE204C20780028BD
:1045B00003D01F48007800282CD00120207000F084
:1045C0003DF81C49152028568A6BA3789206120FD5
:1045D000FF2B00D1A270A278092801DBD21CD2B235
:1045E0000F2A00D90F228B6B3C241207A343920E93
:1045F00013438B630C4C6178012900D072B60028FC
:1046000001DC401E40B26075FDF752FB6078012866
:1046100000D062B66978084A106C1823890798435D
:10462000C90E0843106470BD9012002030120020A3
:10463000AA120020000007408004025010B5444830
:10464000C06AC02108434249C862424880680821C4
:1046500088434049886008468068082188430830BC
:104660003C4988600846C068042188433949C860CD
:104670000846C06804218843001D3649C8600846C2
:10468000C06802218843801C3249C860084680689F
:10469000C008C000401C88600A20FDF76AFF2E4851
:1046A0000078002801D1FDF7E3FA2B4800780028B4
:1046B0000FD1FBF76FFEFDF77FFAFFF7D3FC27481A
:1046C0000078002801D000F0F9FD002000F034FE51
:1046D0002CE02348C06A7F21890388432049C862AF
:1046E0000846C06A7F21490588431E490988890810
:1046F00049057F225205114008431949C8620846FE
:10470000806AFF2149018843174909784901FF223E
:10471000520111400843124988620846806B000A22
:1047200000021249097808430D4988630C4840305B
:10473000C06840084000401C09494031C8600A2058
:10474000FDF717FFFFF7AAFEFFF7B6FE10BD00004A
:104750000000044000000250AA120020B012002005
:1047600000040250CC1200207A6100007861000041
:1047700070B5FEF7ADFD002802D000F0A9FC01E005
:1047800000F070FB7D21FF2289011A48FBF766FDCE
:10479000012149021848FBF768FD1848FFF7CEFCD5
:1047A0001748FBF79FFEFBF73EFDFBF733FD154C6B
:1047B000A07112484089FBF7F3FD134948681C2299
:1047C000904300254860FBF7D3FDE07801280ED127
:1047D0000E4E2078002804D025703178301D00F06E
:1047E00027F86078002803D0E0780128F1D0012074
:1047F00070BD000094180020941600207412002050
:1048000022120020581200200005025090150020AE
:1048100070B505460C46032C00DD70BDA978224614
:104820000248FDF714FD00BFF7E700000004025046
:10483000F8B5974C0E4605460378421CE07895493A
:10484000092B1BD21F007F443F79FF19BF44160478
:1048500017499F16B7DDFE0003228F49681CFBF73E
:104860000FFD00280AD1A0616071FEF71BFF022036
:10487000E070002000F08AF9FBF77AFDF8BD02280D
:10488000FCD10320E0706878A081A978E171E97813
:1048900021720203052149038048FCF76BF8A089C7
:1048A000FA2100030546FBF731FC80B22082002983
:1048B00001D0401C20827D2109012846FBF726FCFF
:1048C00080B2E081002901D0401CE08174A176A073
:1048D000FEF706FA238AE289A18974A0FEF700FA9E
:1048E000F8BD0328FCD1507812780002104340BA7A
:1048F00068496081C308CA5CC108C900471A012120
:10490000B9400A436349C006CA54C00EF11E484369
:104910006C49F21E4018E91CFBF78EFC606960A12F
:104920008019C01E606160A0FEF7DAF961895948FC
:10493000CA08825C64A06369FEF7D2F9608901222B
:10494000C106D206D14203D0218A401C8842C7D179
:104950000520A1697D254003AD0109182B46594A60
:104960004E48FCF7C9FCFF2229465648FBF776FC67
:10497000A0694BA14019A0614BA0FEF7B1F959A065
:104980006269A169FEF7ACF900206061F8BDE289B7
:104990000020002A0DDD01230D5CED432D062D0EB8
:1049A00002D00020A07007E0401CA3709042F3DB0F
:1049B000F8BDA0780028FBD10620E070F8BD0628DD
:1049C000FCD1507812780002104340BAC208C708E0
:1049D0006081FF00C71B8B5C0120B84003438B54F0
:1049E0002FA131A0FEF77CF9F21E618940A0FEF7ED
:1049F00077F96089FA214843052149034118F31EDC
:104A0000EA1C2648FCF778FCF8BD60790028FBD149
:104A10000025A0892E46002823D9012000030090FC
:104A20000520290340030918264B3B221B48FCF7AD
:104A30001FFA0023324801211A46C9024778FB18A1
:104A40008778DBB2BA18D2B2801C00E013E0491EAE
:104A5000F4D198188019C6B26D1CA089ADB28542F8
:104A6000DBD366710EA110A0FEF73AF9617925A09B
:104A7000FEF736F9F8BD592227481623882102602F
:104A8000036001600468002CF9D0FBF7F5FDF8BD68
:104A90005812002094160020B05A00000000054073
:104AA0005B495D200000000025730000706B745F9F
:104AB00074626C5F6E756D2025642C25642C2564F2
:104AC0000A000000941800206368756E6B5F706BBD
:104AD0005F696E6465782025642C25782C25640A2E
:104AE000000000006C656E2025642C25640A00001F
:104AF0007472616E732025642C25640A0000000026
:104B00009318002063616C63756C6174655F7375E5
:104B10006D2025780A000000400003400EB5184AB9
:104B200007CA6B4607C31748406801214904084378
:104B3000144948600846C06940084000C8610846FA
:104B4000C0690121090488430E49C86108464068CC
:104B50000121490488430B4948600B48C069022180
:104B600088430949C8610846C06902218843801CFE
:104B70000549C861002203216846FBF7EDFB0EBD25
:104B8000D85A0000C00402500000025010B504467C
:104B90000348048121460348FDF781FB10BD000056
:104BA000901200200004025030B5C1B00446FF212D
:104BB000013101A8FBF759FB134800680002000A05
:104BC00021780906090E090608430F490860211DCE
:104BD00001A82268FBF730FB00250EE0A80001A920
:104BE00008580A490968491989000122D20389181D
:104BF000074A89180860681CC5B22068C01C800874
:104C0000A842EBD841B030BDC00402502C120020A5
:104C10000000025010B5084CE070A079FFF760FC6E
:104C2000E078042804D0032802D0FCF799FE10BDD8
:104C3000FCF722FF10BD00009012002070B5044662
:104C400021780020012901D0022944D1617802296C
:104C500002D0032919D030E0A178012902D000291F
:104C600009D02AE0E0780021401EC0B200F054F8DC
:104C7000FF21653107E0E0780121401EC0B200F05D
:104C80004BF8FF216131081A17E0A1786E25012940
:104C900002D0002909D010E0E0780021401EC0B207
:104CA00000F03AF8281A80B207E0E0780121401EAF
:104CB000C0B200F031F8281A80B207498A6C430468
:104CC000D20BD2035B0C1A438A64002803D1002163
:104CD0002046FBF76BFB70BD8004025010B5044604
:104CE00060780349487061780248FDF7F2F910BD19
:104CF0009012002000040250064989697F221202A6
:104D00009143044A91611146896902021143014AA3
:104D100091617047C004025030B503460020012B5A
:104D200043D1012920D1002208E09400414D2D6893
:104D30002C59240E2418E0B2541CE2B23E4C2468D4
:104D4000A4089442F1D8002208E094003B4D2D685D
:104D50002C59240E2418E0B2541CE2B2384C2468BA
:104D6000A4089442F1D863E0002208E09400354D95
:104D70002D682C59240E2418E0B2541CE2B2324C97
:104D80002468A4089442F1D8002208E094002F4D32
:104D90002D682C59240E2418E0B2541CE2B22C4C7D
:104DA0002468A4089442F1D842E0012920D10022CD
:104DB00008E094001F4D2D682C59240E2418E0B2F1
:104DC000541CE2B21C4C2468A4089442F1D800227E
:104DD00008E094001F4D2D682C59240E2418E0B2D1
:104DE000541CE2B21C4C2468A4089442F1D81FE081
:104DF000002208E09400134D2D682C59240E24182D
:104E0000E0B2541CE2B2104C2468A4089442F1D8D9
:104E1000002208E09400114D2D682C59240E24180E
:104E2000E0B2541CE2B20E4C2468A4089442F1D8BB
:104E300030BD000010130020CC120020041300200D
:104E4000D812002014130020E0120020F4120020D9
:104E5000C412002000130020D0120020F012002005
:104E6000BC12002010B50024A000714940187149FF
:104E700008607148714902686E480068FBF7DCF908
:104E80006D4800688008001984B2A0006849401885
:104E90006B4908606B486C49026869480068FBF719
:104EA000CBF9684800688008001984B2A000604906
:104EB00040186649086066486649026863480068A9
:104EC000FBF7BAF9624800688008001984B2A000B4
:104ED00057494018604908606048614902685E4867
:104EE0000068FBF7A9F95D4800688008001984B2E2
:104EF000A0004F4940185B4908605B485B49026865
:104F000058480068FBF798F957480068800800196E
:104F100084B2A00046494018554908605548564992
:104F2000026853480068FBF787F952480068800818
:104F3000001984B2A0003E4940185049086050480A
:104F4000504902684D480068FBF776F94C48006804
:104F50008008001984B2A000354940184A49086009
:104F60004A484B49026848480068FBF765F94748DA
:104F700000688008001984B2A0002D4940184549F6
:104F8000086045484549026842480068FBF754F903
:104F9000414800688008001984B2A00024494018E4
:104FA0003F4908603F48404902683D480068FBF7B8
:104FB00043F93C4800688008001984B2A0001C49ED
:104FC00040183A4908603A483A4902683748006848
:104FD000FBF732F9364800688008001984B2A00057
:104FE000134940183449086034483549026832484A
:104FF0000068FBF721F9314800688008001984B285
:10500000A0000B4940182F4908602F482F4902681B
:105010002C480068FBF710F92B480068800800193D
:1050200084B2A010642801DD00BFFEE7204610BD59
:1050300030380020F0120020BC1200205060000028
:10504000F4120020C41200206C600000F81200204E
:10505000C012002088600000FC120020C81200204E
:10506000A460000000130020D0120020D8600000CF
:1050700004130020D8120020F46000000813002060
:10508000D4120020106100000C130020DC1200205C
:105090002C61000010130020CC120020C46000001E
:1050A00014130020E01200204861000018130020B3
:1050B000E4120020546100001C130020E8120020BC
:1050C0005861000020130020EC120020386000001E
:1050D00070B500245E4E30195E4908603119002316
:1050E0001A460420FEF716FB05465B48056060196A
:1050F00084B2301959490860311900231A46062034
:10510000FEF708FB054656480560601984B2301961
:1051100054490860311900231A460820FEF7FAFAAC
:10512000054651480560601984B230194F4908603E
:10513000311900231A460A20FEF7ECFA05464C48BE
:105140000560601984B230194A490860311900239A
:105150001A460520FEF7DEFA054647480560601945
:1051600084B2301945490860311900231A460720D6
:10517000FEF7D0FA054642480560601984B230193E
:1051800040490860311900231A460920FEF7C2FA87
:1051900005463D480560601984B230193B490860F6
:1051A000311900231A460B20FEF7B4FA0546384899
:1051B0000560601984B2301936490860311900233E
:1051C0001A460220FEF7A6FA054633480560601924
:1051D00084B2301931490860311900231A4603207E
:1051E000FEF798FA05462E480560601984B230191A
:1051F0002C490860311900231A460C20FEF78AFA60
:10520000054629480560601984B2301927490860AD
:10521000311900231A460D20FEF77CFA0546244872
:105220000560601984B230192249086031190023E1
:105230001A460F20FEF76EFA05461F4805606019F2
:1052400084B2A010642801DD00BFFEE7204670BDD7
:1052500030380020F0120020BC120020F412002090
:10526000C4120020F8120020C0120020FC120020FE
:10527000C812002000130020D012002004130020C8
:10528000D812002008130020D41200200C13002094
:10529000DC12002010130020CC1200201413002078
:1052A000E012002018130020E41200201C1300203C
:1052B000E812002020130020EC1200201CB51B482F
:1052C0000090002201216846FBF746F8184800903C
:1052D00001AA01216846FBF73FF804210198084321
:1052E00000041349491E084300900022012168462A
:1052F000FBF732F81320009001AA01216846FBF762
:105300002BF8022101980843000412210843009061
:10531000002201216846FBF71FF806480090002292
:1053200001216846FBF718F81CBD000012FF0100C0
:105330001310000012FF000038B504462004044991
:1053400008430090002201216846FBF705F838BDAC
:1053500012FF000010B506A107A0FDF7C1FC07A0D1
:10536000FDF7BEFC41200003FEF78AF810BD0000E7
:105370005B495D2000000000257300004368656301
:105380006B2076616C696420696D61676520696E68
:1053900020417070204261636B757020506172749F
:1053A0006974696F6E2E2E0A0000000010B50F4C54
:1053B0004020616881436160014600222046FCF77D
:1053C0005FF86068610108436060094C042061680F
:1053D00081436160014600222046FCF751F8606875
:1053E000012189040843606010BD000000000240F4
:1053F0004000024010B50F4C002240212046FCF72F
:105400003FF861684020014361600B48FDF7B1F847
:1054100000200A497D23DB008A69012A08D08A69B5
:10542000012A05D0801C80B29842F5D3012010BD1E
:10543000002010BD000002401027000000020240C2
:1054400010B50F4C002204212046FCF719F86168C2
:105450000420014361600B48FDF78BF800200A49E6
:105460007D23DB008A6A012A08D08A6A012A05D0D6
:10547000801C80B29842F5D3012010BD002010BDE1
:1054800040000240102700000002024010B5FFF764
:105490006FF910BD10B5024902A0FDF721FC10BD47
:1054A00060570000257320696E2E2E0A0000000050
:1054B00010B5024902A0FDF713FC10BD755700009E
:1054C000257320696E2E2E0A0000000010B50249D7
:1054D00002A0FDF705FC10BD8A5700002573206966
:1054E0006E2E2E0A0000000070470000C300024824
:1054F000C1501818426070476015002070B5084D03
:105500000024E600A859002805D08047002802D0D2
:10551000701940688047641CE4B2062CF1D370BD5A
:105520006015002010B50446016810A0FDF7D8FBF7
:1055300012A06168FDF7D4FB14A0A168FDF7D0FBB1
:1055400016A0E168FDF7CCFB18A02169FDF7C8FBA8
:105550001AA06169FDF7C4FB1CA0A169FDF7C0FB9F
:105560001EA0E169FDF7BCFB10BD000072302020D9
:105570003D20307825780D0A00000000723120208F
:105580003D20307825780D0A00000000723220207E
:105590003D20307825780D0A00000000723320206D
:1055A0003D20307825780D0A00000000723132204D
:1055B0003D20307825780D0A000000006C72202014
:1055C0003D20307825780D0A00000000706320200F
:1055D0003D20307825780D0A00000000707372209D
:1055E0003D20307825780D0A0000000030B50346D4
:1055F0000024002003E01D5C2C19451CA8B2884241
:10560000F9DB101930BD000010B5592121481622D0
:1056100088230160026003600468002CF9D01E49F1
:105620000A6B012002430A631C4C616A0622114383
:105630006162616A014361620002FBF76FF86069B1
:105640000F2109038843606100210820FBF728F837
:105650006015FAF7B3FFE06940084000E061606957
:105660000F21090488436061606909018843606112
:1056700000212015FAF748FF01211820FAF744FF0E
:105680000121C020FAF740FF032000214003FAF770
:105690003BFF10BD400003400000074000000440F5
:1056A00030B589B00025202001AB0B2241010090CC
:1056B0002848FBF7BBFBFF35FF35023504202649A0
:1056C000088008466946497A81706946897AC170BE
:1056D000002429E00F2C01DB09B030BDA0001E49D9
:1056E000085AA1001C4A891849884018C01C81B278
:1056F000601C8000115220200090601C8000105A15
:1057000001229202811801AB0B221248FBF78EFB9B
:10571000601C8000104940186946497981706946CB
:105720008979C170601CC4B2A0000B49085AA1005D
:10573000094A891849884018C01C08490988091D68
:105740008842C7DB002001E0411CC8B21028FBDB07
:1057500000BFC1E700000540F037002028130020FB
:10576000736C6565705F74696D6572305F68616EDA
:10577000646C657200736C6565705F74696D6572E9
:10578000315F68616E646C657200736C6565705F33
:1057900074696D6572325F68616E646C6572000079
:1057A000127D00001362000002FF00001262000080
:1057B00002FF0000126203000256800002B30C00D8
:1057C00002B4000002B5000002BE000002B60000F4
:1057D00002B7000012B8000002FF00000200000043
:1057E00002020802020A0864020398FF0203900002
:1057F000020A00001202000002FF0000020204027E
:10580000020A0814022D24FF022D0400020A0000DF
:1058100012020000020300000212200002272000F2
:10582000127D0000D7AE240013C624008BF42400A0
:105830007BFF240073422500275F25005B90250035
:105840006DAE25008FC1250021CB2500B2D42500E7
:105850000256800002B30C0002B4000002B5000042
:1058600002BE000002B6000002B7000012B800003D
:10587000027D000002030000021220001227200017
:1058800002FF01000220320002228800029F1A005B
:1058900002560200021E3E00021F2000020FE2011B
:1058A0000201400112FF000000100E000300000082
:1058B00000002110422063308440A550C660E7708C
:1058C000088129914AA16BB18CC1ADD1CEE1EFF134
:1058D0003112100273325222B5529442F772D662DC
:1058E000399318837BB35AA3BDD39CC3FFF3DEE384
:1058F0006224433420040114E664C774A44485542C
:105900006AA54BB528850995EEE5CFF5ACC58DD5D3
:105910005336722611163006D776F6669556B4467B
:105920005BB77AA719973887DFF7FEE79DD7BCC723
:10593000C448E5588668A7784008611802282338CB
:10594000CCC9EDD98EE9AFF9488969990AA92BB973
:10595000F55AD44AB77A966A711A500A333A122A1B
:10596000FDDBDCCBBFFB9EEB799B588B3BBB1AABC3
:10597000A66C877CE44CC55C222C033C600C411C6B
:10598000AEED8FFDECCDCDDD2AAD0BBD688D499D13
:10599000977EB66ED55EF44E133E322E511E700EBB
:1059A0009FFFBEEFDDDFFCCF1BBF3AAF599F788F63
:1059B0008891A981CAB1EBA10CD12DC14EF16FE143
:1059C0008010A100C230E32004502540467067607B
:1059D000B9839893FBA3DAB33DC31CD37FE35EF393
:1059E000B1029012F322D2323542145277625672CB
:1059F000EAB5CBA5A89589856EF54FE52CD50DC5E3
:105A0000E234C324A014810466744764245405441A
:105A1000DBA7FAB79987B8975FE77EF71DC73CD732
:105A2000D326F2369106B01657667676154634566A
:105A30004CD96DC90EF92FE9C899E9898AB9ABA982
:105A40004458654806782768C018E1088238A328BA
:105A50007DCB5CDB3FEB1EFBF98BD89BBBAB9ABBD2
:105A6000754A545A376A167AF10AD01AB32A923A0A
:105A70002EFD0FED6CDD4DCDAABD8BADE89DC98D22
:105A8000267C076C645C454CA23C832CE01CC10C5A
:105A90001FEF3EFF5DCF7CDF9BAFBABFD98FF89F72
:105AA000176E367E554E745E932EB23ED10EF01EAA
:105AB0004F54410001000000010000000000000000
:105AC0009C38D509027D1300027D1D00027D09006E
:105AD000027D1800027D0E0002700E00027A140092
:105AE00012000800024B8000024C500002945B0040
:105AF0000296640002F9A000122E290002FF0000A5
:105B0000027D13000200040002021002020A061EB7
:105B100002FF010002001100020091FA02001100D0
:105B200002FF000002C3BF00027FC10002FF0100AC
:105B30000206000002070300029E00000200185047
:105B400002001000029E0100020018500200100026
:105B5000029E02000200185002001000029E030084
:105B6000020018500200100002FF0000020A0000AC
:105B70000202000002C38F00027FC000127D0000FD
:105B8000B0001900A000000AA000010AA0001178CE
:105B9000A0001301B0001B02B0001B0004E0000ACB
:105BA00014E0030A02FF000002090500025304008A
:105BB00002594000026F2200022B200002780C00E4
:105BC0000279010002700C00022802000262030048
:105BD0000266500002D5000002DF050002DE570019
:105BE00002C4140002C1090002D3790002908900A6
:105BF00002980200028C400002A2060002A30A00E2
:105C000002A30B0002A30A0002A3000002A2D60016
:105C100002A3000002A3010002A3000002A2C2002E
:105C200002A3020002A3030002A3020002A2B70023
:105C300002A3040002A3050002A3040002A20600BE
:105C400002A30C0002A30D0002A30C0002A2F200AA
:105C500002A30E0002A30F0002A30E0002A2DE00A8
:105C600002A3100002A3110002A3100002A2D4009C
:105C700002A3120002A3130002A3120002A2030057
:105C800002A3140002A3150002A3140002A207003D
:105C900002A3160002A3170002A3160002A20F001F
:105CA00002A3180002A3190002A3180002A22F00E9
:105CB00002A31A0002A31B0002A31A0002DAD300F7
:105CC00002DBFA0002D9060002D9070002D9060059
:105CD00002DA0F0002DB750002D90A0002D90B00BC
:105CE00002D90A0002DA000002DB130002D9000028
:105CF00002D9010002D9000002DA000002DB0A002A
:105D000002D9020002D9030002D9020002DAE2003D
:105D100002DBF70002D9040002D9050002D9040011
:105D200002DAE60002DB8C0002D9080002D9090081
:105D300002D9080002DAFB0002DBF20002D90C00F3
:105D400002D90D0002D90C0002DA000002DB80004B
:105D500002D9100002D9110002D9100002DA0000A5
:105D600002DB350002D9120002D9130002D9120059
:105D700002DAE00002DBCF0002D9140002D91500DC
:105D800002D9140002DAC40002DBEB0002D91600CB
:105D900002D9170002D9160002DAE10002DBD900AD
:105DA00002D9180002D9190002D9180002DA1B0022
:105DB00002DB580002D91A0002D91B0002D91A00CE
:105DC00002DAF40002DB400002D91C0002D91D00F7
:105DD00002D91C0002DA040002DBC00002D9200054
:105DE00002D9210002D9200002DA000002DBB5004E
:105DF00002D9220002D9230002D9220002DAE000EF
:105E000002DB670002D9240002D9250002D9240050
:105E100002DAC20002DB840002D9260002D9270080
:105E200002D9260002DAE00002DBFF0002D92800D6
:105E300002D9290002D9280002DA1D0002DB8D00F8
:105E400002D92A0002D92B0002D92A0002DAEE0078
:105E500002DBD00002D92C0002D92D0002D92C007F
:105E600002C94600023B4800029A5200029908000B
:105E700002F4160002F1020002BF0600022A20000E
:105E800002D422000283330002842000027FC0007B
:105E900002AF80000293B00002FF01000220320036
:105EA00002228800029F3A0002560200021E3E00B3
:105EB000021F200002FF000002FF00000231D40098
:105EC0000232380002B9000002BAF00002BB000042
:105ED000022D020002400700023EC00002FF010046
:105EE000020FE2010201400102FF0000020208026B
:105EF000020A08640203088F02030000020A00007D
:105F00000202000002020402020A0814022E00002B
:105F1000022F4D00022D24DF022D0400020A000092
:105F20000202100002022800024B01000229230095
:105F30000295090002F53F0002FF01000200110076
:105F40000200510002007100029E03000200F150A5
:105F50000200110002020800029E000002FF000081
:105F60000295070002F50000024B00000229200004
:105F700002FF000002020A1E0241205802410000F6
:105F8000027E03000241205802410000027E82008E
:105F90000241208802410000027E0200020004004B
:105FA00002021002020A061E02FF01000200110096
:105FB000020091FA0200110002FF000002C3BF00BC
:105FC000027FC10002FF0100020600000207030079
:105FD000029E00000200185002001000029E010004
:105FE0000200185002001000029E02000200185029
:105FF00002001000029E0300020018500200100070
:1060000002FF0000020A00000202000002C38F002B
:10601000027FC0000295010012FF000002FF000095
:1060200002020402020A0814022D24FF022D0400B9
:10603000020A0000120210000200081A020A0824D4
:1060400002004800027A94000274010012701C20C1
:10605000027E020002C2A00002000800020A080A32
:1060600002004800027A940012701410027E0300AD
:1060700002C2A00002000800020A080A020048004A
:10608000027A940012701410027E020002C2E00034
:1060900002000800020A080002004800027A940088
:1060A00012701410027FC100027E220102C2A00001
:1060B00002000800020A08240200481A027A94002A
:1060C00012701410027FC100027FC00002700C1514
:1060D00002000800120A00000262030002700C00B5
:1060E000027E020002C2A00002C3BF0002002C0216
:1060F000120A06190262030002700C00027E0301FC
:1061000002C2A00002C3BF0002002C02120A06193C
:106110000262030002700C00027E020002C2E00074
:1061200002C3BF0002002C02120A061E0262030014
:1061300002700C00027E820102C2280002C3BE006F
:1061400002002C02120A061E026200000228000051
:1061500012000800126E240A020A00001200000059
:10616000040000001400000004000000080000000B
:10617000040000001C0000007D6085030902050387
:10618000092626760800000032640100000700009E
:1061900000010700010000090000000107000100E4
:1061A000000C0000000107000100000800000001D1
:1061B00003000100000F0000000000000100000FBC
:1061C00000000001000001000007000001010700BD
:1061D000010000090000010107000100000A0000A1
:1061E000010105000100000B000001010000010099
:1061F00000070000020107000100000A0000020180
:1062000007000100000A0000020000000100000F6A
:106210000000020000000100000800000300000070
:106220000100000D00000300000001000007000055
:10623000040000000100000C000004000000010048
:106240000009000005000000010000080000060031
:1062500000000100000C0000060000000100000B1F
:106260000000070000000100000B00000800000013
:106270000100000B00000900000001000008000000
:106280000B0000000100000A00000C0000000100EB
:10629000000A00000D0000000100000A01000600D5
:1062A00000000100000801000700000001000008D4
:1062B00001000800000001000007010009000000C3
:1062C00001000009030005000000010000090700AB
:1062D00005000000010000080F000500000001009B
:1062E0000009030007000000010000090700070083
:1062F0000000010000080F00070000000100000975
:106300001F0007000000010000097F0007000000D7
:1063100001000009FF01070000000301000A03005B
:10632000070000000301000C070007000000030144
:1063300000090F00070000000300000C0F00070019
:1063400000000300000D1F00070000000300000B09
:106350007F000700000003000009FF0307000000A2
:106360000300000CFF030700000007000009FF0303
:10637000070000000700000FFF03070000000000F7
:1063800002B9010002BA100012BB000002B90100FC
:1063900002BA100012BB000002561B0002B3080034
:1063A00002B4000002B5000002BE000002B6000008
:1063B00002B7100012B80000021000000211C00065
:1063C000026A800002C94600123B480002C6000172
:1063D00002C7AD0102C8FC01021000000211D20088
:1063E000126A5C0002C94600123B480002DE070048
:1063F000021020000211F200026A200002D90001FE
:1064000002C6000102C7C50102C8D10102C90600C7
:10641000123B7F0002DE0700021020000211F20092
:10642000026A200002D8010002D9400102C603011D
:1064300002C7C00112C8000102C90600123B7F005A
:1064400002700E1A027A140012000800138600006F
:106450001385000012F1000012F10D00122B040050
:1064600013B0000013B10000122B00009C64000068
:10647000000000209C100000322D00003875000044
:106480009C1000209802000000030000DC75000052
:10649000341300208C2E0000422D0000401E2DD30E
:1064A00000BF00BF00BF00BF00BF00BF00BF00BFF4
:1064B00000BF00BF00BF00BF00BF00BF00BF00BFE4
:1064C00000BF00BF00BF00BF00BF00BF00BF00BFD4
:1064D00000BF00BF00BF00BF00BF00BF00BF00BFC4
:1064E00000BF00BF00BF00BF00BF00BF00BF00BFB4
:1064F00000BF00BF00BF00BF401ED1D2704710B523
:10650000134CA069800308D5A06901214904084300
:1065100010490840A06100F0A9FFA069400308D518
:10652000A0690121890408430B490840A06100F0DB
:10653000A3FFA069000308D5A0690121C90408438D
:1065400006490840A06100F09DFF00F0A1FF10BDCA
:1065500000000740E1FFF3FFE1FFF5FFE1FFF9FF76
:10656000401E02D300BF401EFCD27047F0B5F9496F
:1065700083B0CA69C8148243CA61F74C2168CF0747
:106580002168FF0F4906CE0F21690905C90F009147
:1065900021688907C90F0191F049496CF04D01420A
:1065A00011D0606880060ED460684004FCD50120DC
:1065B00000F014FF00220221EA4800F083FD686821
:1065C000002800D08047E5480121406C490208427C
:1065D00024D06068000721D40098304301D0002FF8
:1065E0000AD160684004FCD5012000F0F7FE0022CB
:1065F0000221DC4800F066FDDB49DC484A681018DF
:10660000006802B201208003101AC217920F1018FE
:1066100080104870A868002800D08047CF4801212A
:10662000406C090308421FD0606800061CD46068F3
:106630004004FCD5012000F0D1FE00220221C9480F
:1066400000F040FDC848C9494268511809680AB2BB
:1066500001218903511ACA17920F511889104170EC
:10666000E868002800D08047BC490120496C8006BA
:10667000014211D0606840020ED460684004FCD52D
:10668000012000F0ABFE00220221B64800F01AFD06
:106690002869002800D08047B0480121406C490695
:1066A000084211D0606800020ED460684004FCD536
:1066B000012000F093FE00220221AA4800F002FD12
:1066C0006869002800D08047606880040ED5606843
:1066D00040060BD460684004FCD5002F02D1012095
:1066E00000F07CFEA869002800D080479B4801216B
:1066F000406C890208421BD06068C00618D400981C
:10670000304306D0002E02D00198002801D1002F7E
:106710000AD060680004FCD5012000F05FFE002272
:106720000221904800F0CEFC2868002800D0804765
:106730008A48416CFF2201321143416403B0F0BD2D
:1067400014E78B48C16B49084900C1638948016857
:106750004908490001604168490849004160C72073
:1067600000BF401EFCD270478148C26B01210A4322
:10677000C263804802680A43026042680A4342607A
:106780001D2000BF401EFCD2704770B57B4C7A4D77
:106790009AB02146688118314EC90291214605966A
:1067A0000493039228314EC90996089307920691E3
:1067B0006978012900D072B6064641094901411A9B
:1067C000C9B24009102901D31F3800E02038C3B2F4
:1067D000102900D3203901229204002901DD080389
:1067E00001E00803801802991B04194302918303F6
:1067F0009B0F03991B041943030403911B0E049977
:106800001B041943049100060599000A01430591F0
:10681000E87803280DD004280BD0052809D0361AB3
:1068200070094001301AC0B2102804D371091F3911
:1068300003E0761EF4E771092039C9B2102800D3AD
:106840002038002801DD000301E000038018069ACB
:1068500009040A4306928203920F07991204114316
:1068600002040791120E08991204114308910006C0
:106870000999000A014309910022082102A800F0A9
:1068800065FCE87803284ED004284CD005284AD06F
:1068900086193B4830184F2802D23A48864244D1E4
:1068A0003348C26B01210A43C263324802680A437B
:1068B000026042680A43426000BF00BF1B2000BF65
:1068C000401EFCD211212068490408430090002298
:1068D0000121684600F03AFC204638300FC80AAE65
:1068E0000FC6204648300FC80FC6002208210AA84C
:1068F00000F02CFC00BF00BFC52000BF401EFCD232
:10690000204658300FC812AE0FC6226FE16EA06E3F
:106910001892179116900022072112A800F016FC79
:10692000FFF70FFF3CE0761CB3E7A87A4B21134C2E
:106930004901401A23467433A26F616FE46FDB682C
:10694000C0B20A910C940D930B92C1071CD0400861
:106950001DE0000000000540C00402508004025009
:10696000D437002000040250301200200080025072
:10697000000007404000074090120020A057000090
:106980009EF6FFFFA60900004008401EC0B219464F
:10699000000401430D91002204210AA800F0D6FB57
:1069A0006878012800D062B61AB070BD30B40823F0
:1069B000401E491E521E447855786C404C708478B5
:1069C0009578801C6C408C70891C921C5B1EF2D1E7
:1069D00030BC7047F0B40022082301460F26B51AD8
:1069E0000C78475D0F70491C521C44555B1EF6D154
:1069F000F0BC7047F8B58B4A84468B4D8B4B8C4E60
:106A00008C4C8D4F10683F6836682D6824681B6871
:106A1000401C0DD1A8681060D868506098699060DB
:106A2000B069D060E0681061A0695061B869906198
:106A30006046C078012802D002281ED03AE0002922
:106A400007D05068D860906898611068A860D068D6
:106A500011E0D8680002000AD8609869010201209C
:106A6000090AC00608189861A8680002000AA86010
:106A7000B0690002000AB0611CE0002907D010696B
:106A8000E0605069A0611068A860906911E0E0685A
:106A90000002000AE060A06901020120090AC006A4
:106AA0000818A061A8680002000AA860B86900027E
:106AB000000AB86100F0DCFBF8BD10B55F4C0022A5
:106AC0000221204600F0FEFA002000F087FC01229F
:106AD0000221204600F0F6FA10BDF7B5002482B07E
:106AE000064627460094012901D0022903D100213E
:106AF0003046FFF77FFF5148806A8003C50EB078AB
:106B0000002835D1F0784E49012802D0022818D04B
:106B100069E02C4618204443096808342046890857
:106B20004C43317801295ED146490A340968890805
:106B3000491C484304190020012100F0AFFC0090DB
:106B400016E02C461820444309680834204689087A
:106B50004C433178012946D13B490A3409688908F8
:106B6000491C484304190120014600F097FC00909D
:106B7000B078012837D1F1783448012902D00229B0
:106B800019D030E018212C464C43006808342146C7
:106B90008008444330780B27012824D12C480A343C
:106BA00000688008401C41430C190020014600F099
:106BB00075FC009017E018212C464C4300680834FF
:106BC0002146800844433078052701280BD121480D
:106BD0000A3400688008401C41430C190120002140
:106BE00000F05CFC0090B17860090129049913D091
:106BF000091A0098081A401F00B200280ADB3178F1
:106C0000012907D114498A6C4304D20BD2035B0CCF
:106C10001A438A6405B0F0BD091A0098081AC01B0F
:106C2000401EE9E73812002010130020F012002067
:106C300000130020F412002004130020000402506E
:106C4000CC120020D0120020D8120020E012002028
:106C5000BC120020C412002080040250F0B5FFB026
:106C6000FFB093B00022FFA90A6343224A620122C7
:106C70008A620022CA624864002101E0002808D02C
:106C8000FFA89C4A436AD06F8007C017401CFAD106
:106C900013607D20984BC002DA6B120702D4401EAD
:106CA000FAD131E0934800680004000C2CD401288C
:106CB00006D0022806D004280BD0182824D116E0CC
:106CC000802401E00124A402FFA9496A43294ED08F
:106CD00050E088480622C16F8907C917491CFAD1BC
:106CE0000260FFA8C06A7FB07FB013B0F0BD7D2006
:106CF0008002DA6B120702D4401EFAD104E07D480C
:106D0000006880B2182821D0FFA8491C406A0229D7
:106D1000B4DB432827D077481822C16F8907C917E9
:106D2000491CFAD102601822C16F8907C917491C92
:106D3000FAD102601822C16F8907C917491CFAD11C
:106D400002607FB07FB0881E13B0F0BD6949062293
:106D5000C86F8007C017401CFAD10A607FB07FB0AF
:106D6000401E13B0F0BD1520FFA9486284E7012141
:106D7000FFAA11630021FFAA516269460872FFA8A9
:106D800002AA006B01320025002800D00120001962
:106D9000C01C002819DD7D26564FB6023046D96B3F
:106DA000090702D4401EFAD199E038680004000CAB
:106DB0004FD41070FFA8006B521C6D1C002800D02F
:106DC00001200019C01CA842E8DC6846477A807A96
:106DD000C043C0B287423CD1FFA8806A874204D03A
:106DE000FFA8806A401E874279D1FFA802A9006BE4
:106DF00003318C4600282DD0084600222146002C65
:106E00001DDD401ECB0704D0427853003B4A401C96
:106E1000D25A611013D0394D130A467812027340CA
:106E20005B00EB5A867853409AB2130A73405B00BA
:106E3000EB5A12025340801C9AB2491EECD16046B4
:106E40006146005D091949780002401880B282420B
:106E500026D044E00020631E002B16DD0122E5074A
:106E6000D207491ED54201D04878491C4D780022EE
:106E70005B1008D08E784019CD789219891CC0B269
:106E8000D2B25B1EF6D18018C0B2611E0A0003D4D4
:106E90006146895C0818C0B26146095D81421ED115
:106EA000FFA8806A874208D1FFA9486CC96A2246B8
:106EB000401802A9033100F0F7FAFFA8C06A0119CF
:106EC000FFA8C162806A401CC1B2FFA88162094864
:106ED0000622C16F8907C917491CFAD106E0054887
:106EE0001522C16F8907C917491CFAD10260002118
:106EF000CFE600000030004040300040B0580000B5
:106F000070B5C2B0284800F055F8274D002628601B
:106F10002879264C012803D0042801D0267117E0D7
:106F20000A21A07900F0C6FA2079814203D000F04E
:106F3000C7FAFFF7C2FD2079401CC0B220710A28B1
:106F400000D326712979684601290CD0042916D06E
:106F5000287907281DD00096684600F0B7FA01206E
:106F6000207042B070BD291D001D2A6800F0B4FADF
:106F7000A079694608722868401C0090ECE705215A
:106F80000171E2890A49401D00F0ACFAE089401C19
:106F900007E0072168460171A1794171617981712A
:106FA00003200090D8E70000901500205812002020
:106FB0009416002030B5C1B00446FF21013101A86C
:106FC00000F096FA39480068394940180068000214
:106FD000000E206020788007800F002802D12068F2
:106FE000850802E020688008451C00200CE0820033
:106FF0002E490968091D51182D4A8918096882000F
:1070000001AB9950411CC8B2A842F0D301A9201D80
:10701000226800F061FA207841B030BD10B501213E
:10702000244800F06BFA00F0E3F910BD10B50446F7
:10703000204600F069FA6089FFF7A7FBFFF73DFDE6
:1070400010BD38B51C48C078052805D10121194864
:1070500000F060FA002800D138BD72B6684600F032
:107060005FFA164900980968884204D313490098CA
:107070000968401A06E0114800680021C943081A4F
:1070800000994018044662B660017D21C90000F0F5
:1070900011FA04460A48844205D900F047FA00F084
:1070A0000FFAFFF70AFD00BFD6E7000034120020F8
:1070B000008002500004025090120020AC12002008
:1070C000A0611C0010B502291BD1002A0CD0DC23C2
:1070D0001B5801242343DC242350DC231B58CC03FE
:1070E0002343DC2423502FE0DC231B585C0864007E
:1070F000DC231C501B5801242404A343DC2423500C
:1071000022E000290FD1002A06D0DC231B580124DD
:107110002343DC24235017E0DC231B585C08640065
:10712000DC231C5010E0002A07D0DC231B5801246C
:1071300024042343DC24235006E0DC231B580124D1
:107140002404A343DC24235010BD0000FCB50346F7
:1071500000250195009500240020002900D186E03B
:1071600000BFAA4DAD6A6D086D006D1CA74EB562DB
:107170003546AD6A6D086D00B5623546AD6A0226CA
:10718000B543AD1CA14EB5623546AD6A0226B54386
:107190009E4EB56200BF3546AD6A1026B543103528
:1071A0009A4EB56200BF00BF984DAD6A0126F60445
:1071B0003540ED0C0195019D012DF5D0934D2D6BC2
:1071C0002646641CB6009E593546904E35633546BA
:1071D000AD6A0126760535406D0D0195002A08D06F
:1071E000019D002D05D1894D6D6B0646401CB600F2
:1071F00095518C42D7D300BF009D6D1C0095834DE7
:1072000040356D68ED07ED0F0195019D002DF3D020
:107210007E4DAD6A0126760535406D0D01950CE079
:107220007A4D6D6B0646401CB6009551774DAD6AA0
:107230000126760535406D0D0195002A02D0019D8D
:10724000002DEDD0714D4035AD686D086D006D1CA1
:107250006E4E4036B5603546AD686D086D00B56060
:107260006A4DAD6A1026B543684EB56200BFFCBDDD
:10727000002100200120000300BF08E08A00644BC9
:107280001B689A58634BC3181A60001D491C624A58
:10729000126892088A42F1D8002108E08A005F4B08
:1072A0001B689A585B4BC3181A60001D491C5C4A46
:1072B000126892088A42F1D8002108E08A00594BEE
:1072C0001B689A58534BC3181A60001D491C564A34
:1072D000126892088A42F1D8002108E08A00534BD4
:1072E0001B689A584B4BC3181A60001D491C504A22
:1072F000126892088A42F1D84E4AD278042A03D002
:107300004C4AD278032A0FD1002108E08A004A4B68
:107310001B689A583F4BC3181A60001D491C474A06
:10732000126892088A42F1D8002108E08A00444B92
:107330001B689A58374BC3181A60001D491C414AF4
:10734000126892088A42F1D8002108E08A003E4B78
:107350001B689A582F4BC3181A60001D491C3B4AE2
:10736000126892088A42F1D8324AD278042A03D0AD
:10737000304AD278032A10D1002108E08A00344B29
:107380001B689A58234BC3181A60001D491C314AC8
:10739000126892088A42F1D81FE0002108E08A00B2
:1073A0002D4B1B689A581B4BC3181A60001D491CB3
:1073B0002A4A126892088A42F1D8002108E08A001D
:1073C000274B1B689A58134BC3181A60001D491CA1
:1073D000244A126892088A42F1D8704710B50446D0
:1073E000002C02D1FFF7C0F901E0FFF7AAF910BDA8
:1073F00000B589B020221C4901A800F06DF80022D8
:10740000082101A8FFF7A2FE09B000BD0004025048
:107410001013002000000250CC1200201413002092
:10742000E0120020F0120020BC120020F412002014
:10743000C412002090120020F8120020C012002078
:1074400000130020D012002004130020D8120020C6
:1074500008130020D4120020FC120020C8120020C3
:107460000C130020DC1200209863000003B40148D4
:10747000019001BD9554000003B40148019001BD85
:10748000B154000003B40148019001BDCD54000087
:1074900003B40148019001BDE954000003B4014860
:1074A000019001BD194D000003B40148019001BDD8
:1074B000B536000003B40148019001BD0D01000084
:1074C00003B40148019001BD1D4B000003B4014805
:1074D000019001BDA94B000003B40148019001BD1A
:1074E0003902000003B40148019001BD39020000D7
:1074F00003B40148019001BD6B02000003B40148D0
:10750000019001BDD320000003B40148019001BDEA
:10751000DD4C000003B40148019001BD0D210000C5
:1075200003B40148019001BDAD37000003B4014828
:10753000019001BD2D4100009201A2FF121002181E
:107540004089302132037A02340A170134B20A32F8
:107550000982080A188068D169310A184064D1721A
:107560000D0A255030720E8A30907C030203DB0135
:107570001432053A043489640C1B03020C34320BB8
:10758000021C0A827D22FF1A10061901011D1A0130
:107590000209161B1D030102021F1550C3CE095814
:1075A0000801050471764129342119192B020109BA
:1075B0001B6209CA291C5A761A9113127D1B017885
:1075C000E1321C690432209A14106904320C192B20
:0C75D0001132080237182940C1000000E9
:04000005000000F106
:00000001FF
